:020000040800F2
:1000000000060020F50500086135000819350008D4
:10001000413500081935000839350008F705000892
:10002000F7050008F7050008F70500084545000832
:10003000F7050008F7050008F7050008F7050008B0
:10004000F7050008F7050008F7050008F7050008A0
:10005000F7050008F70500086575000891750008A8
:10006000BD750008E975000815760008F705000859
:10007000F7050008F7050008F7050008F705000870
:10008000F7050008F7050008F7050008C93400085F
:10009000F1340008DD340008053500084176000819
:1000A000F7050008F7050008F7050008F705000840
:1000B000F7050008F7050008F7050008F705000830
:1000C000F7050008F7050008F7050008F705000820
:1000D000F7050008F7050008F7050008F705000810
:1000E000A5760008F7050008F7050008F7050008E1
:1000F000F7050008F7050008F7050008F7050008F0
:10010000F7050008F70500082D770008F705000837
:10011000F7050008F7050008F7050008F7050008CF
:10012000F7050008F7050008F7050008F7050008BF
:10013000F7050008F7050008F7050008F7050008AF
:10014000F7050008F7050008F7050008F70500089F
:10015000F7050008F7050008F7050008F70500088F
:10016000F7050008F7050008F7050008F70500087F
:10017000F7050008ED6B0008F7050008F705000813
:10018000F7050008F705000819770008F7050008CB
:10019000F7050008F7050008F7050008F70500084F
:1001A000F7050008F7050008F7050008F70500083F
:1001B000F7050008F7050008F7050008F70500082F
:1001C000F7050008F7050008F7050008F70500081F
:1001D000F7050008D96B0008F7050008F7050008C7
:1001E000F7050008F7050008F7050008F7050008FF
:1001F000F7050008F7050008F7050008F7050008EF
:10020000F7050008F7050008F7050008F7050008DE
:10021000F7050008F7050008F7050008F7050008CE
:10022000F7050008F7050008F7050008F7050008BE
:10023000F7050008F7050008F7050008F7050008AE
:10024000F7050008F7050008F7050008F70500089E
:10025000F7050008F7050008F7050008F70500088E
:10026000F7050008F7050008F7050008F70500087E
:10027000F7050008F7050008F7050008F70500086E
:10028000F7050008F7050008F7050008F70500085E
:10029000F7050008F7050008F7050008F70500084E
:1002A000F7050008F7050008F7050008F70500083E
:1002B000F7050008F7050008F7050008F70500082E
:1002C000F7050008F7050008F7050008F70500081E
:1002D000F7050008F7050008F7050008F70500080E
:1002E000111A0008000000000000000000000000DB
:1002F00053B94AB9002908BF00281CBF4FF0FF318D
:100300004FF0FF3000F074B9ADF1080C6DE904CE88
:1003100000F006F8DDF804E0DDE9022304B07047E0
:100320002DE9F047089D04468E46002B4DD18A42A8
:10033000944669D9B2FA82F252B101FA02F3C2F1DB
:10034000200120FA01F10CFA02FC41EA030E94406C
:100350004FEA1C48210CBEFBF8F61FFA8CF708FB8D
:1003600016E341EA034306FB07F199420AD91CEB65
:10037000030306F1FF3080F01F81994240F21C8197
:10038000023E63445B1AA4B2B3FBF8F008FB1033DF
:1003900044EA034400FB07F7A7420AD91CEB040414
:1003A00000F1FF3380F00A81A74240F207816444E4
:1003B000023840EA0640E41B00261DB1D440002369
:1003C000C5E900433146BDE8F0878B4209D9002DCD
:1003D00000F0EF800026C5E9000130463146BDE857
:1003E000F087B3FA83F6002E4AD18B4202D38242C1
:1003F00000F2F980841A61EB030301209E46002D70
:10040000E0D0C5E9004EDDE702B9FFDEB2FA82F2C4
:10041000002A40F09280A1EB0C014FEA1C471FFA22
:100420008CFE0126200CB1FBF7F307FB131140EA09
:1004300001410EFB03F0884208D91CEB010103F1D6
:10044000FF3802D2884200F2CB804346091AA4B298
:10045000B1FBF7F007FB101144EA01440EFB00FE6C
:10046000A64508D91CEB040400F1FF3102D2A645D1
:1004700000F2BB800846A4EB0E0440EA03409CE770
:10048000C6F12007B34022FA07FC4CEA030C20FA1D
:1004900007F401FA06F31C43F9404FEA1C4900FA3D
:1004A00006F3B1FBF9F8200C1FFA8CFE09FB1811BA
:1004B00040EA014108FB0EF0884202FA06F20BD92D
:1004C0001CEB010108F1FF3A80F08880884240F27D
:1004D0008580A8F102086144091AA4B2B1FBF9F0C1
:1004E00009FB101144EA014100FB0EFE8E4508D9BC
:1004F0001CEB010100F1FF346CD28E456AD9023841
:10050000614440EA0840A0FB0294A1EB0E01A14225
:10051000C846A64656D353D05DB1B3EB080261EB93
:100520000E0101FA07F722FA06F3F1401F43C5E96D
:10053000007100263146BDE8F087C2F12003D840A3
:100540000CFA02FC21FA03F3914001434FEA1C47E5
:100550001FFA8CFEB3FBF7F007FB10360B0C43EAD7
:10056000064300FB0EF69E4204FA02F408D91CEB87
:10057000030300F1FF382FD29E422DD90238634485
:100580009B1B89B2B3FBF7F607FB163341EA034125
:1005900006FB0EF38B4208D91CEB010106F1FF3874
:1005A00016D28B4214D9023E6144C91A46EA00466B
:1005B00038E72E46284605E70646E3E61846F8E6FD
:1005C0004B45A9D2B9EB020864EB0C0E0138A3E746
:1005D0004646EAE7204694E74046D1E7D0467BE727
:1005E000023B614432E7304609E76444023842E79F
:1005F000704700BF02E000F000F8FEE772B637482F
:1006000080F30888364880F3098836483649086000
:1006100040F20000CCF200004EF63471CEF2000140
:100620000860BFF34F8FBFF36F8F40F20000C0F23E
:10063000F0004EF68851CEF200010860BFF34F8FF4
:10064000BFF36F8F4FF00000E1EE100A4EF63C71E1
:10065000CEF200010860062080F31488BFF36F8F8C
:1006600005F030FD06F03EFD4FF055301F491B4AA6
:1006700091423CBF41F8040BFAE71D49184A9142E8
:100680003CBF41F8040BFAE71A491B4A1B4B9A423C
:100690003EBF51F8040B42F8040BF8E7002018495C
:1006A000184A91423CBF41F8040BFAE705F048FDB7
:1006B00006F09CFD144C154DAC4203DA54F8041BB3
:1006C0008847F9E700F042F8114C124DAC4203DACA
:1006D00054F8041B8847F9E705F030BD00060020F8
:1006E000002200200000000808ED00E000000020CB
:1006F00000060020E07C000800220020D02200201C
:10070000D022002030870020E0020008E402000828
:10071000E4020008E40200082DE9F04F2DED108AF4
:10072000C1F80CD0D0F80CD0BDEC108ABDE8F08F29
:10073000002383F311882846A047002004F0AAFF75
:10074000FEE704F003FF00DFFEE70000F8B501F06C
:1007500075F905F03BFC074605F0AAFC0546B8BB59
:10076000204B9F4234D001339F4234D027F0FF0208
:100770001D4B9A4232D12E4642F21074F8B200F06C
:1007800093FF00F097FF08B10024264601F04CFDCE
:1007900020B10024032000F07BF8264635B1134B2E
:1007A0009F4203D0002405F07BFC2646002005F084
:1007B00017FC0EB100F082F801F0E2FA00F0AEFF93
:1007C00001F0B8F9204600F029F900F077F8F9E7D0
:1007D0002E460024D5E704460126D2E7064641F21C
:1007E0008834CEE7010007B0000008B0263A09B00F
:1007F00008B501F06BF9A0F120035842584108BD3B
:1008000007B541F21203022101A8ADF8043001F04E
:100810007BF903B05DF804FB38B5302383F311880E
:10082000174803680BB105F001F80023154A4FF48F
:100830007A71134804F0F0FF002383F31188124CFF
:10084000236813B12368013B2360636813B16368B5
:10085000013B63600D4D2B7833B963687BB902208F
:1008600001F010FA322363602B78032B07D1636801
:100870002BB9022001F006FA4FF47A73636038BD99
:10088000D022002019080008F0230020E8220020D0
:10089000084B187003280CD8DFE800F008050208A0
:1008A000022001F0EDB9022001F0E8B9024B00226C
:1008B0005A607047E8220020F0230020F8B501F0CC
:1008C000B3FC30B14D4B03221A7000224C4B5A60DE
:1008D000F8BD4C4B4C4A1C4619680131F8D0043322
:1008E0009342F9D16268494B9A42F1D9484B9B68CF
:1008F00003F1006303F500339A42E9D205F0A4FB4B
:1009000005F0B6FB002001F02FF90220FFF7C0FF31
:10091000404B0021D3F8E820C3F8E810D3F81021A9
:10092000C3F81011D3F81021D3F8EC20C3F8EC1061
:10093000D3F81421C3F81411D3F81421D3F8F020FC
:10094000C3F8F010D3F81821C3F81811D3F8182100
:10095000D3F8802042F00072C3F88020D3F88020C2
:1009600022F00072C3F88020D3F8803072B64FF0C6
:10097000E023C3F8084DD4E90004BFF34F8FBFF361
:100980006F8F254AC2F88410BFF34F8F536923F449
:1009900080335361BFF34F8FD2F8803043F6E07657
:1009A000C3F3C905C3F34E335B0103EA060C2946C2
:1009B0004CEA81770139C2F87472F9D2203B13F105
:1009C000200FF2D1BFF34F8FBFF36F8FBFF34F8F65
:1009D000BFF36F8F536923F4003353610023C2F8D0
:1009E0005032BFF34F8FBFF36F8F302383F31188E3
:1009F000854680F3088820476AE700BFE822002088
:100A0000F02300200000020820000208FFFF010878
:100A1000002200200044025800ED00E02DE9F04FD4
:100A200093B0B74B2022FF2100900AA89D6801F0E7
:100A300051F9B44A1378A3B90121B3481170036086
:100A4000302383F3118803680BB104F0EFFE002319
:100A5000AE4A4FF47A71AC4804F0DEFE002383F313
:100A60001188009B13B1AA4B009A1A60A94A137807
:100A7000032B03D000231370A54A53604FF0000AE4
:100A8000009CD3465646D146012001F0F9F824B126
:100A90009F4B1B68002B00F02C82002001F016F801
:100AA0000390039B002B01DA00F08CFE039B002BCC
:100AB000EDDB012001F0E2F8039B213B1F2BE3D883
:100AC00001A252F823F000BF490B0008710B000887
:100AD000050C0008890A0008890A0008890A00082C
:100AE000970C0008670E0008810D0008E30D000850
:100AF0000B0E0008310E0008890A0008430E00089A
:100B0000890A0008B50E0008E90B0008890A0008E8
:100B1000F90E0008550B0008E90B0008890A0008C7
:100B2000E30D0008890A0008890A0008890A0008FC
:100B3000890A0008890A0008890A0008890A000849
:100B4000890A0008050C00080220FFF751FE002862
:100B500040F0F981009B022105A8BAF1000F08BFFF
:100B60001C4641F21233ADF8143000F0CDFF8BE794
:100B70004FF47A7000F0AAFF071EEBDB0220FFF7AC
:100B800037FE0028E6D0013F052F00F2DE81DFE8C6
:100B900007F0030A0D1013360523042105A8059359
:100BA00000F0B2FF17E004215548F9E704215A4844
:100BB000F6E704215948F3E74FF01C08404608F1D6
:100BC000040800F0D3FF0421059005A800F09CFF65
:100BD000B8F12C0FF2D101204FF0000900FA07F70D
:100BE00047EA0B0B5FFA8BFB01F0C0F826B10BF064
:100BF0000B030B2B08BF0024FFF702FE44E7042180
:100C00004748CDE7002EA5D00BF00B030B2BA1D14D
:100C10000220FFF7EDFD074600289BD001200026AB
:100C200000F0A2FF0220FFF733FE1FFA86F84046CD
:100C300000F0AAFF0446B0B1039940460136A1F185
:100C400040025142514100F0B7FF0028EDD1BA46B1
:100C5000044641F21213022105A83E46ADF81430B5
:100C600000F052FF10E725460120FFF711FE244B4C
:100C70009B68AB4207D9284600F078FF013040F06E
:100C800067810435F3E70025224BBA463E461D70C6
:100C90001F4B5D60A8E7002E3FF45CAF0BF00B0329
:100CA0000B2B7FF457AF0220FFF7F2FD322000F04C
:100CB0000DFFB0F10008FFF64DAF18F003077FF409
:100CC00049AF0F4A08EB0503926893423FF642AFE3
:100CD000B8F5807F3FF73EAF124BB845019323DD57
:100CE0004FF47A7000F0F2FE0390039A002AFFF6A8
:100CF00031AF039A0137019B03F8012BEDE700BFE9
:100D000000220020EC230020D02200201908000837
:100D1000F0230020E82200200422002008220020E6
:100D20000C220020EC220020C820FFF761FD0746BE
:100D300000283FF40FAF1F2D11D8C5F120020AABD8
:100D400025F0030084494245184428BF42460192D9
:100D500000F09AFF019AFF217F4800F0BBFF4FEAA5
:100D6000A803C8F387027C492846019300F0BAFF24
:100D7000064600283FF46DAF019B05EB830533E782
:100D80000220FFF735FD00283FF4E4AE00F026FF17
:100D900000283FF4DFAE0027B846704B9B68BB428B
:100DA00018D91F2F11D80A9B01330ED027F0030347
:100DB00012AA134453F8203C05934046042205A987
:100DC000043701F01BFA8046E7E7384600F0CEFE14
:100DD0000590F2E7CDF81480042105A800F094FEF8
:100DE00002E70023642104A8049300F083FE002896
:100DF0007FF4B0AE0220FFF7FBFC00283FF4AAAE60
:100E0000049800F0E1FE0590E6E70023642104A8C1
:100E1000049300F06FFE00287FF49CAE0220FFF7E1
:100E2000E7FC00283FF496AE049800F0CFFEEAE716
:100E30000220FFF7DDFC00283FF48CAE00F0DEFE60
:100E4000E1E70220FFF7D4FC00283FF483AE05A9B8
:100E5000142000F0D9FE07460421049004A800F0F5
:100E600053FE3946B9E7322000F030FE071EFFF688
:100E700071AEBB077FF46EAE384A07EB0903926888
:100E800093423FF667AE0220FFF7B2FC00283FF422
:100E900061AE27F003074F44B9453FF4A5AE48467D
:100EA00009F1040900F062FE0421059005A800F094
:100EB0002BFEF1E74FF47A70FFF79AFC00283FF41D
:100EC00049AE00F08BFE002844D00A9B01330BD0C2
:100ED00008220AA9002000F005FF00283AD02022AD
:100EE000FF210AA800F0F6FEFFF78AFC1C4804F078
:100EF000D7FB13B0BDE8F08F002E3FF42BAE0BF004
:100F00000B030B2B7FF426AE0023642105A8059369
:100F100000F0F0FD074600287FF41CAE0220FFF72A
:100F200067FC804600283FF415AEFFF769FC41F2EC
:100F3000883004F0B5FB059800F062FF46463C4659
:100F400000F014FFA0E506464EE64FF0000901E66A
:100F5000BA467EE637467CE6EC22002000220020DE
:100F6000A0860100094A49F26900136899B21B0C76
:100F700000FB013344F250611360054B186882B2E4
:100F8000000C01FB0200186080B2704714220020A0
:100F9000102200200021102210B5044600F09AFE15
:100FA000034B03CB206061601868A06010BD00BFD8
:100FB00000E8F11F2DE9F041ADF5507D0D4600210F
:100FC00040F275126EAC074610A80F9100F082FE39
:100FD0004FF4C4720021204600F07CFE0DF13C0865
:100FE00002F0C6FA4FF47A72264BB0FBF2F01860AA
:100FF00093E80700022384E807000DF5ED702382D3
:10100000FFF7C8FF47F605031F4907A8238406F02A
:1010100031FC1F230DF2EB220DF1340C84F8323138
:1010200007AB1E46083203CE664542F8080C42F86C
:10103000041C3346F5D1306810602046B188B3797E
:10104000918041469371012200F0FCFE002380B2A2
:10105000E97E0393AB7E029305F11903019301230B
:10106000009306A3D3E90023CDE90480384602F0BB
:101070003DFE0DF5507DBDE8F08100BF9E6AC421A4
:10108000818A46EEF8230020847800082DE9F0419B
:101090002C4CDAB080460D46237A5BBB27A9284644
:1010A00000F0DEFF0746002842D19DF89D60C82E63
:1010B0003ED801464FF4A662204600F00BFE4FF4E6
:1010C000807332460DF19E01C4F8F8314FF400737D
:1010D00004F109002644C4F80C334FF44073C4F8FB
:1010E000203400F0D1FD9DF89C30777223720BB94B
:1010F000EB7E237206AC8122002127A800F0EAFDD6
:101100000122214627A800F0E7FF002380B2E97EF4
:101110000393AB7E029305F1190301932823CDE9D4
:1011200004400093404605A3D3E9002302F0DEFD0E
:101130005AB0BDE8F08100BFAFF300802641727263
:10114000DF25D7B7A05D0020F0B5254E4FF48A7596
:10115000F1B0002405FB006596F8D830D82221466E
:1011600085F8DC303AA885F8E84006AF00F0B2FD1B
:1011700006F1090000F0A6FDD5F8E430C2B206F190
:1011800009018DF8F0000DF1F100CDE93A3400F0DD
:101190007BFD394601223AA800F0CAFF082380B23D
:1011A000317ACDE9047001270E48CDE9023706F106
:1011B000D80301933023009307A3D3E9002302F05F
:1011C00095FDA04206DD02F0D3F9C5F8E0003846EF
:1011D00071B0F0BD2046FBE778F6339F93CACD8D02
:1011E000A05D0020103400202DE9F04F274F87B07C
:1011F000DFF8A480264E384602F0A4FD03460028FE
:101200003CD00024234DADF81440A1460294A246E0
:10121000CDE90344027B8DF8142003AA9968406845
:1012200003C21B6843F0004302932B6804F22C5462
:10123000D3F810B002F09EF910EB0802CDF800A030
:10124000284605F5A55541F1000302A9D84740F607
:1012500058230028C8BF49F0010910359C42E4D149
:10126000B9F1000F05D0384602F070FD86F800A0F5
:10127000C1E73378072B04D80133337007B0BDE8DA
:10128000F08F024802F062FDF8E700BF1034002042
:10129000D56200204034002040420F0070B50D465A
:1012A00014461E4602F07EFC50B9022E10D1012CCD
:1012B0000ED112A3D3E900230120C5E9002307E0E2
:1012C000282C10D005D8012C09D0052C0FD00020D7
:1012D00070BD302CFBD10BA3D3E90023ECE70BA3AB
:1012E000D3E90023E8E70BA3D3E90023E4E70BA34A
:1012F000D3E90023E0E700BFAFF30080401DA12049
:1013000026812A0B78F6339F93CACD8D9E6AC4211D
:10131000818A46EE26417272DF25D7B7F017304A30
:1013200039059E5638B505460E4C0021013500F0B2
:1013300043FCA4F82C55B4F82C0500F025FC78B13A
:10134000B4F82C0500F030FC014648B9B4F82C057F
:1013500000F032FCB4F82C350133A4F82C35EAE760
:1013600038BD00BFA05D0020F8B50E4C02260E4F20
:10137000A4F5805343F8307C237E3BB965692DB1D9
:10138000284600F0CBFF284606F02AFA2046A4F5AE
:10139000A55400F0C3FF012EA4F1100400D1F8BD44
:1013A0000126E5E720590020447900082DE9F04F97
:1013B0008FB005460C4600AF02F0F4FB002849D17F
:1013C000237E022B1BD1E38A012B18D102F0D0F827
:1013D0000646FFF7C7FD03464FF4C87006F51676BC
:1013E000DFF8C082B3FBF0F202FB103316FA83F38E
:1013F000C8F80030E37E33B9A34B00221A703C37A3
:10140000BD46BDE8F08F07F12401204600F0E6FD5F
:101410000028F4D107F11400FFF7BCFD97F826402F
:1014200007F1140107F12700224606F0F1F9002820
:10143000E2D10F2C08D8944B1C70D8F80030A3F5DB
:101440001673C8F80030DAE797F82410284602F03F
:10145000A1FBD4E7E38A282B2BD010D8012B23D073
:10146000052BCCD1BFF34F8F8849894BCA6802F452
:10147000E0621343CB60BFF34F8F00BFFDE7302B1B
:10148000BDD1844EE17E327A9142B8D1607E314640
:10149000002291F8DC50854200F0A580013201F570
:1014A0008A71042AF5D1AAE721462846FFF782FD72
:1014B000A5E721462846FFF7E9FDA0E7B2F8EC5082
:1014C0007B6005F103094FEA99094FEA8902D11DB2
:1014D000C908A8EBC10300219D46EB46584600F021
:1014E000F9FB04F1EE012A465846314400F0CCFBEA
:1014F0007B6813B9012000F037FB96F8D20000F0AA
:1015000043FB044630B9307200F068FB204600F01F
:101510002BFBB1E0D6F8D4203AB996F8D200B6F851
:101520002C25824201D8FFF7FDFED6F8D4202A44AC
:10153000944208D296F8D200B6F82C2501308242A7
:1015400001D8FFF7EFFE5FFA89F25946706800F0A4
:10155000C9FB08B9C54679E0726896F8D2002A44FA
:101560007260D6F8D42005EB0209C6F8D49000F0DA
:101570000BFB814509D396F8D220D6F8D40001326E
:10158000001B86F8D220C6F8D400FF2D0FD8002407
:10159000347200F023FB204600F0E6FA00F044FE2F
:1015A0003D4B188108B9FFF789F9C54627E7BB68A5
:1015B00096F8D9000AFB0362FB68D2F8E41082F8BF
:1015C000E83001F58061C2F8E030C2F8E410FFF7BE
:1015D000BBFDFFF709FE96F8D920013202F00302A5
:1015E00086F8D920B6E74FF48A7A20460AFB02F53E
:1015F00005F1EA01314400F0C7FDF86000287FF4EE
:10160000FEAE0122354485F8E82001F0B1FFD5F89F
:10161000E020D6ED007A801A40F6B832B8EE677A4C
:10162000DFED1E6A192838BF1920904228BF1046E6
:1016300007EE900AF8EEE77A67EEA67ADFED186A11
:10164000E7EE267AFCEEE77AC6ED007A96F8D93016
:10165000BB60BA6873680AFB02F4321992F8E810AA
:1016600059B1D2F8E410E8468B423FF427AF00218D
:1016700082F8E810C2F8E010C5467368064A9B0A73
:1016800001331381BBE600BF0934002000ED00E008
:101690000400FA05A05D0020F8230020CDCCCC3D4D
:1016A0006666663F0C340020014B1870704700BF1F
:1016B0000424002038B54FF04054144B22689A425D
:1016C00021D1627D0025124B12481A70C922237D58
:1016D0000930114900F8013C4FF48073C0F8DB5029
:1016E000C0F8EF314FF40073C0F803334FF4407388
:1016F000C0F8173400F0C8FAE0222946204600F06E
:10170000E9FA012038BD0020FCE700BF9AAD44C5CE
:1017100004240020A05D00201600003037B500F042
:1017200083FD1F4C1F4D022301221F496B7123684B
:101730002881204604F580545B6898470122D4F83C
:10174000B03404F5966018495B6898470023174940
:101750004FF480520193164B16480093164B02F03B
:10176000F1F9164B197811B1124802F013FA01F091
:10177000FFFE0446FFF7F6FB4FF4C873B0FBF3F22D
:1017800002FB130304F5167010FA83F00C4B18607B
:1017900004F08EFC08B10F232B8103B030BD00BFD5
:1017A00040340020F823002040420F00082400208D
:1017B0009D12000810340020AD13000804240020FE
:1017C0000C3400202DE9F04F00252DED028B93B055
:1017D0000DF12C084FF0010ADFF814B2FFF704FDF9
:1017E0000A95ADF834500B95C8F804509FED798BED
:1017F00000267E4C374623680DF11D0207A92046BE
:101800008DF81CA08DF81D508DED008BD3F808903D
:101810000023C8479DF81C90B9F1000F1ED010227C
:1018200000210EA800F056FA236808AA0AA95F69E9
:1018300020460DF11E03B8470FAB4F4698E8030052
:1018400083E803009DF834300EA958468DF84430E3
:101850000A9B0E93DDE9082302F056FC06F22C5693
:1018600040F6582304F5A5549E4204F11004C2D159
:10187000002FBDD15E4802F095F900283FD15D4EA2
:1018800001F076FE3368984239D301F071FE0446C8
:10189000FFF768FB4FF4C8738DF82870B0FBF3F2C4
:1018A00002FB130304F5167010FA83F03060524EF9
:1018B000377817B901238DF82830C7F110040EA826
:1018C000FFF768FB0EABE4B20DF12900D919062C25
:1018D00028BF06242246013400F0D6F90AABE4B250
:1018E00043480393182304940293444B0193012328
:1018F00000933AA3D3E9002302F09AF9357001F07E
:1019000037FE3F4A3F4C1368C31AB3F57A7F2FD393
:10191000106001F02FFE02460B46354802F020FA17
:10192000334802F03FF918B3237A0EAF364E002B3E
:1019300014BF03230223737101F01AFE4FF47A736C
:1019400001223946B0FBF3F03060304600F01EFB58
:10195000182380B202932D4B019340F25513CDE929
:101960000370009322481FA3D3E9002302F060F91B
:10197000237A93B101F0FCFD002607464FF48A78E4
:1019800094F8D900304400F0030008FB004393F8BA
:10199000E82072B10136042EF2D1C82003F080FE97
:1019A000237A002B7FF414AF13B0BDEC028BBDE89B
:1019B000F08FD3F8E02042B12368BA1AFA2B38BF6F
:1019C000FA230533B2EB430FE4D3FFF7BDFB002846
:1019D000E0D1E2E70000000000000000401DA1206F
:1019E00026812A0BF1C6A7C1D068080F4034002019
:1019F000103400200C34002009340020083400206A
:101A0000D0620020A05D0020F8230020D4620020D6
:101A100008B5064801F0B6F8054801F0B3F8054AE4
:101A200005490020BDE8084005F0D4BE4034002040
:101A3000F048002030630020691300087047000060
:101A40002DE9F84F4FF47A7306460D46002402FB49
:101A500003F7DFF85080DFF8509098F900305FFA14
:101A600084FA5A1C01D0A34212D159F824002A4604
:101A700031460368D3F820B03B46D847854207D1AA
:101A8000074B012083F800A0BDE8F88F0124E4E7AC
:101A9000002CFBD04FF4FA7003F002FE0020F3E7B5
:101AA0001C630020182200201C22002070B5044670
:101AB0004FF47A76412C254628BF412506FB05F0D8
:101AC00003F0EEFD641BF5D170BD0000002307B5E7
:101AD000024601210DF107008DF80730FFF7B0FF36
:101AE00020B19DF8070003B05DF804FB4FF0FF3014
:101AF000F9E700000A46042108B5FFF7A1FF80F0CE
:101B00000100C0B2404208BD074B0A4630B4197804
:101B1000064B53F82140014623682046DD69044BFB
:101B2000AC4630BC604700BF1C6300201C22002074
:101B3000A086010070B50A4E00240A4D04F0CCF8CE
:101B4000308028683388834208D904F0C1F82B68B4
:101B500004440133B4F5003F2B60F2D370BD00BFE5
:101B60001E630020D862002004F084B900F10060F8
:101B700000F500300068704700F10060920000F549
:101B8000003004F005B90000054B1A68054B1B88AE
:101B90009B1A834202D9104404F09AB8002070477F
:101BA000D86200201E630020024B1B68184404F01A
:101BB00095B800BFD8620020024B1B68184404F09F
:101BC0009FB800BFD86200200020704700F1FF508E
:101BD00000F58F10D0F8000870470000064991F812
:101BE000243033B100230822086A81F82430FFF73B
:101BF000C3BF0120704700BFDC620020014B1868A2
:101C0000704700BF0010005C194B013803220844E4
:101C100070B51D68174BC5F30B042D0C1E88A6422A
:101C20000BD15C680A46013C824213460FD214F97C
:101C3000016F4EB102F8016BF6E7013A03F10803B8
:101C4000ECD181420B4602D22C2203F8012B042452
:101C5000094A1688AE4204D1984284BF967803F8A8
:101C6000016B013C02F10402F3D1581A70BD00BFB0
:101C70000010005C24220020D0780008704700008B
:101C80007047000070470000002310B5934203D056
:101C9000CC5CC4540133F9E710BD0000013810B525
:101CA00010F9013F3BB191F900409C4203D11AB1B8
:101CB0000131013AF4E71AB191F90020981A10BDE8
:101CC0001046FCE703460246D01A12F9011B002910
:101CD000FAD1704702440346934202D003F8011B35
:101CE000FAE770472DE9F8431F4D1446074688462A
:101CF00095F8242052BBDFF870909CB395F82430FF
:101D00002BB92022FF2148462F62FFF7E3FF95F809
:101D100024004146C0F1080205EB8000A24228BF22
:101D20002246D6B29200FFF7AFFF95F82430A41BED
:101D300017441E449044E4B2F6B2082E85F824609D
:101D4000DBD1FFF74BFF0028D7D108E02B6A03EB6C
:101D500082038342CFD0FFF741FF0028CBD1002080
:101D6000BDE8F8830120FBE7DC620020024B1A7813
:101D7000024B1A70704700BF1C630020182200201D
:101D800038B51A4C1A4D204602F0A8FF29462046C5
:101D900002F0D0FF2D684FF47A70D5F89020D2F879
:101DA000043843F00203C2F80438FFF77FFE1149FC
:101DB000284603F0CDF8D5F890200F4DD2F804381E
:101DC000286823F002030D49A042C2F804384FF4FA
:101DD000E1330B6001D002F0DFFE6868A04204D05E
:101DE0000649BDE8384002F0D7BE38BD106A002071
:101DF000707A0008787A00081C2200200463002012
:101E00000C4B70B50C4D04461E780C4B55F8262033
:101E10009A420DD00A4B002118221846FFF75AFFAC
:101E20000460014655F82600BDE8704002F0B4BEDB
:101E300070BD00BF1C6300201C220020106A00201F
:101E4000046300202DE9F0470D460446002190462A
:101E5000284640F27912FFF73DFF23462022002159
:101E6000284604F1220702F0F1F8231D0222202166
:101E70002846C02602F0EAF8631D032222212846E4
:101E800002F0E4F8A31D03222521284602F0DEF823
:101E900004F1080310222821284602F0D7F804F1A3
:101EA000100308223821284602F0D0F804F111036B
:101EB00008224021284602F0C9F804F11203082242
:101EC0004821284602F0C2F804F1140320225021D0
:101ED000284602F0BBF804F118034022702128467E
:101EE00002F0B4F804F120030822B021284602F0E1
:101EF000ADF804F121030822B821284602F0A6F823
:101F0000314608363B4608222846013702F09EF843
:101F1000B6F5A07FF4D1002704F1330A04F13203AF
:101F200008223146284602F091F894F832304FEA00
:101F3000C7099F4209F5A47615D3B8F1000F08D15F
:101F4000314609F24F1604F599730722284602F02C
:101F50007DF827463B1B94F8322193420CD3F01DA9
:101F6000C008BDE8F0870AEB07030822314628467F
:101F7000013702F06BF8D8E707F233133146082235
:101F800028460836013702F061F8E3E713B5044646
:101F9000084600212022234601900160C0F803106A
:101FA00002F054F8231D01980222202102F04EF87D
:101FB000631D01980322222102F048F8A31D019815
:101FC0000322252102F042F8019804F108031022AF
:101FD000282102F03BF8072002B010BD0023F7B51E
:101FE0000E46047F072200911946054601F0F2FED5
:101FF000731C0122072100932846002301F0EAFE0A
:10200000C4B9B31C052208212846009323460D2499
:1020100001F0E0FE3746BB1BB278934211D3073480
:102020002B7FA88AE408BBB9844294BF002001201A
:1020300003B0F0BDAB8A0824DB00083BDB08B370BB
:10204000E8E7FB1C214608222846009300230834B9
:10205000013701F0BFFEDEE7201A18BF0120E7E7D5
:102060000023F7B50E46047F082200911946054665
:1020700001F0B0FE731CC4B908220093234610245B
:102080001146284601F0A6FE01235F1C7278013B31
:10209000934211D307342B7FA88AE408BBB984424A
:1020A00094BF0020012003B0F0BDAB8A0824DB0000
:1020B000083BDB087370E7E7F3192146082228463E
:1020C0000093002301F086FE08343B46DDE7201A2A
:1020D00018BF0120E7E70000F8B50E460546144694
:1020E000002181223046FFF7F5FD2B460822002112
:1020F000304601F0ABFF7CB90F246B1C072208218E
:10210000304601F0A3FF01235F1C6A78013B934234
:1021100004D3E01DC008F8BD0824F4E7EB192146FC
:102120000822304601F092FF08343B46ECE70000FD
:10213000F8B50E46054614460021CE223046FFF77C
:10214000C9FD2B4628220021304601F07FFF7CB9D3
:10215000302405F1080308222821304601F076FFDB
:102160002F467B1B2A7A934204D3E01DC008F8BD9A
:102170002824F5E707F109032146082230460834F0
:10218000013701F063FFECE7F7B5047F0E460091DD
:10219000012310220021054601F01CFEC4B9B31C26
:1021A00009221021284600932346192401F012FE2B
:1021B00037467288BB1B9A4211D807342B7FA88AF6
:1021C000E408BBB9844294BF0020012003B0F0BDF5
:1021D000AB8A1024DB00103BDB087380E8E73B1D73
:1021E000214608222846009300230834013701F0D5
:1021F000F1FDDEE7201A18BF0120E7E730B50A44F9
:10220000084D91420DD011F8013B5840082340F38E
:102210000004013B2C4013F0FF0384EA5000F6D188
:10222000EFE730BD2083B8EDF7B5364A6B4610684E
:1022300051686A4603C308233349344805F0F8FA65
:10224000044690BB0A25324A6B46106851686A46BC
:1022500003C308232F492D4805F0EAFA0446002855
:1022600047D00369B3F5F01F43D8B0F86620B2F544
:10227000AF6F3ED1284A024402F15C018B4238D351
:102280005C3B224900209E1AFFF7B8FF04F164016D
:10229000074632460020FFF7B1FFA3689F4228D1CE
:1022A000E368984208BF002523E00369B3F5F01FF7
:1022B00026D8428BB2F5AF6F20D1174A024402F103
:1022C00010018B4218D3103B104900209D1AFFF7D4
:1022D00095FF04F1180106462A460020FFF78EFFFD
:1022E000A3689E4202D1E368984201D00D25AAE777
:1022F0000025284603B0F0BD1025A4E70C25A2E771
:102300000B25A0E7E0780008DCFF1D0000000208B4
:10231000E978000890FF1D000800FEF710B5037C67
:10232000044613B9006805F06BFA204610BD0000A2
:102330000023BFF35B8FC360BFF35B8FBFF35B8F83
:102340008360BFF35B8F7047BFF35B8F0068BFF3A1
:102350005B8F704770B505460C30FFF7F5FF0446FC
:1023600005F108063046FFF7EFFFA04206D96D6879
:102370003046FFF7E9FF2544281A70BD3046FFF7C5
:10238000E3FF201AF9E7000070B505464068A0B1E8
:1023900005F10C0605F10800FFF7D6FF04463046AC
:1023A000FFF7D2FF844204F1FF34304694BF6D68DA
:1023B0000025FFF7C9FF2C44201A70BD38B50C4624
:1023C0000546FFF7C7FFA04210D305F10800FFF74D
:1023D000BBFF04446868BFF35B8FB4FBF0F100FB04
:1023E00011440120AC60BFF35B8F38BD0020FCE7D7
:1023F0002DE9F041144607460D46FFF7C5FF84421C
:1024000028BF0446D4B1B84658F80C6B4046FFF7D5
:102410009BFF3044286040467E68FFF795FF331AE3
:102420009C4203D801206C60BDE8F081A41B6B6066
:102430003B682044AB60E8600220F5E72046F3E704
:1024400038B50C460546FFF79FFFA04210D305F1B3
:102450000C00FFF779FF04446868BFF35B8FB4FB9F
:10246000F0F100FB11440120EC60BFF35B8F38BD3D
:102470000020FCE72DE9FF418846694607466C4687
:10248000FFF7B6FF002506B204EBC606B4420AD039
:10249000626808EB050120680834FFF7F5FB54F883
:1024A000043C1D44F2E729463846FFF7C9FF284699
:1024B00004B0BDE8F0810000F8B505460C300F46C9
:1024C000FFF742FF05F1080604463046FFF73CFFE0
:1024D000A042304688BF6C68FFF736FF201A38608C
:1024E00020B12C683046FFF72FFF2044F8BD0000D4
:1024F00073B5144606460D46FFF72CFF8442019043
:1025000028BF0446DCB101A93046FFF7D5FF019B87
:1025100033B93268C5E90233C5E9002401200CE073
:102520009C42286038BF0194019884426860F5D9C4
:102530003368241A0220AB60EC6002B070BD204604
:10254000FBE700002DE9FF410F4669466C46FFF7A7
:10255000CFFF00B2002604EBC005AC4209D0D4F88E
:102560000480B81954F8081B42464644FFF78CFB18
:10257000F3E7304604B0BDE8F081000038B5054609
:10258000FFF7E0FF044601462846FFF717FF204605
:1025900038BD0000302383F3118862B67047000015
:1025A000002383F3118862B6704700000120704752
:1025B0007047000010B41346026814680022A44655
:1025C0005DF8044B6047000000F5805090F8590416
:1025D0007047000000F5805090F8520470470000EA
:1025E00000F5805090F95804704700004E20704765
:1025F00000F5805208B5FFF7CDFFD2F89834D2F835
:1026000094041844D2F890341844D2F8783418441A
:10261000D2F888341844D2F884341844FFF7C0FF45
:1026200008BD00002DE9F04F0C4600F5805185B043
:102630001F4691F8523405469046BDF838909BB13C
:10264000D1F874340133C1F8743423689A0006D485
:10265000237B082B0BD9627B0AB10F2B07D9D1F84A
:1026600078340133C1F878344FF0FF300FE0FFF7D2
:1026700091FFEB6AD3F8C42012F4001A0AD0D1F803
:102680007C3400200133C1F87C34FFF789FF05B0AA
:10269000BDE8F08F22684FF0480BD3F8C460002AE1
:1026A0006B6AC6F30446B4BF42F0804292041BFB3F
:1026B000063BCBF8002023685B004FEA066344BF6B
:1026C00042F00052CBF80020227B43EA0243720121
:1026D000CBF80430607B18B343F44013CBF80430DC
:1026E000D1F8A4340133C1F8A434AB1803F58353F3
:1026F000197B41F020011973207B039200F094FFB5
:102700000330039A80105FFA8AF30AF1010A8342C8
:102710000DDA04EB83010BEB830349689960F2E760
:10272000AB1803F58353197B60F34511E3E70121EF
:10273000EB6A04F10C00B140C3F8D010AB1821468D
:1027400003F58253C3E9048705EB461303F582536F
:10275000183351F804CB814243F804CBF9D10988EE
:102760002A442846198041F26803D65002F5805267
:1027700009F0030392F86C1043F0100321F01F01DD
:102780000B43214682F86C304246FFF709FF3B4677
:10279000CDF8009000F00EFF012078E72DE9F0471A
:1027A00000F58056044696F85254002D40F0018101
:1027B000037C032B40F092802B4628462F465FFA7D
:1027C00083FC944510DA01EBCC0E51F83CC0BCF10F
:1027D000000F04DBDEF804C0BCF1000F02DB0137A0
:1027E0000133ECE70130FBE7FFF7D4FEE36AF0B911
:1027F000D3F8800040F00200C3F880004E23E06A66
:10280000002F6ED1D0F8803043F00103C0F8803043
:10281000694B6A4A1B6803F1805303F52C539B00F4
:102820009342A36240F2AF80654800F09BFE4D28C2
:1028300042D8DFF884814FEA004EDFF88891D8F85B
:1028400000C04EEA8C0EC3F884E00CF1805303F50F
:102850002C539B00636100EB0C03D4F82CC0C8F828
:102860000030C0F14E03DCF8800040F03000CCF8BE
:1028700080004FF0000CD4F81480E6465FFA8CF02C
:102880008242BCDD01EBC00A51F83000002810DBA9
:10289000DAF804A0BAF1000F0BDA09EA00400AF0F6
:1028A0007F0A40EA0A0040F0084048F82E000EF186
:1028B000010E0CF1010CE1E79A6922F001029A6124
:1028C00000F056FE0646E36A9B69D90704D500F07E
:1028D0004FFE831BFA2BF6D9FFF762FE2846BDE8B0
:1028E000F087B7EB530F3DD2DFF8CCE04FEA074C4F
:1028F000DEF800304CEA830CC0F888C003F1805049
:1029000003EB4703002700F52C50CEF80030BC46FF
:102910008000A061E06AD0F8803043F00C03C0F87A
:102920008030D4F818E0FBB29A427FF771AF51F8CB
:10293000330001EBC3080028D8F8043001DB002B7A
:102940000EDB20F0604023F0604340F0005043F085
:1029500000434EF83C000EEBCC000CF1010C436040
:102960000137E0E7836923F00103836100F000FE93
:102970000646E36A9B69DA07AED500F0F9FD831BD2
:10298000FA2BF6D9A8E7E26A936923F00103936171
:1029900000F0EEFD0746E36A9B69DB0705D500F012
:1029A000E7FDC31BFA2BF6D996E7012586F85254AA
:1029B00092E7002592E700BF2C630020FCB50040A1
:1029C000F47800080000FF0713B500F5805401916A
:1029D000606CFFF7D9FC1F280AD920220199606C8E
:1029E000FFF748FDA0F120035842584102B010BD46
:1029F0000020FBE700F5805008B5FFF7CBFD406CE9
:102A0000FFF796FCBDE80840FFF7CABD0022026050
:102A100082814260826070470022002310B5C0E9C5
:102A20000023002304460C3020F8043CFFF7EEFF9F
:102A3000204610BD2DE9F047074688B09A468846E3
:102A400007F5805468469146FFF7A4FDFFF7E4FFC1
:102A5000606CFFF77FFC1F282DD920226946606C2F
:102A6000FFF78CFD202826D194F852341BB303AD18
:102A7000444605AB2E46083403CE9E4244F8080C6B
:102A800044F8041C3546F5D130684146206038468C
:102A9000B388A380DDE90023C9E90023BDF808302D
:102AA0004A46AAF80030FFF77BFD534608B0BDE860
:102AB000F04700F06DBD0020FFF772FD08B0BDE8E3
:102AC000F08700002DE9F84F0023064600F58154F9
:102AD000054688461034C0E90133274B46F8303BA1
:102AE000374638462037FFF797FFA742F9D105F55B
:102AF00080544FF4805305F5A3594FF0000A266324
:102B00000026676405F5835709F110094FF0000BA3
:102B10001037E663C4E90D36012384F8403084F8A9
:102B20004830A7F11800203747E910ABFFF76EFFD8
:102B300047F8286C4F45F4D1B8F1010F84F8588458
:102B4000A4F85A64A4F85C64A4F85E6484F8606431
:102B5000A4F86264A4F86464A4F8666484F8686401
:102B600002D9064800F0FEFC054B284653F82830F1
:102B7000EB62BDE8F88F00BF4479000818790008BF
:102B800034790008044B10B5197804464A1C1A70B1
:102B9000FFF798FF204610BD296300202DE9F0477C
:102BA00000295FD0304F3148B7FBF1F581428CBF2F
:102BB0000A201120431EB5FBF0FC00FB1C50DCB2C8
:102BC00020B1022B1846F5D8002037E00CF1FF3574
:102BD000B5F5806F32D2C4EBC4094FF47A7009F1B5
:102BE00003034FEAE308C3F3C70308F1010AA4EBA8
:102BF000030E08FB00085FFA8EF65AFA8EFEB8FB49
:102C0000FEFEBEF5617F1BDC1FFA8EF4581C56FADF
:102C100080F00CFB00FCB7FBFCFC6145D4D1013B10
:102C2000DBB20F2BD0D8711E0020C9B2072905D8FE
:102C3000107101201480558053719171BDE8F087A7
:102C400009F1FF334FEAE30EC3F3C7030EF10108A6
:102C5000E41A0EFB0000E6B258FA84F4B0FBF4F478
:102C6000A4B2D3E70846E9E700B4C4043F420F002A
:102C700038B540F27772C36A154CC3F8BC200722FE
:102C8000C36AC3F8C8202268C16A930043F4C02312
:102C9000C1F8A03002F1805302F16C01C56A03F55E
:102CA0002C53EA3289009B00226041F0E061094A1E
:102CB000C361C5F8C01003F5D87103F56A734162AA
:102CC0009342836202D9044800F04CFC38BD00BF37
:102CD0002C630020FCB50040F47800082DE9F04F8B
:102CE00000F58055994689B0044695F858348A46CF
:102CF0009046022B04D90027384609B0BDE8F08F72
:102D00009B4A52F8231009B942F823009949C4F8A4
:102D10000CA00B7884F81090C3B9FFF73BFC964BDE
:102D2000D3F8EC2042F48072C3F8EC20D3F894205E
:102D300042F48072C3F89420D3F8942022F4807275
:102D4000C3F8942001230B70FFF72AFC95F8513447
:102D50006BB9FFF71FFC894A95F85834D35CEBB187
:102D6000012B24D0012385F85134FFF719FCFFF71C
:102D700011FCE26A936923F01003936100F0F8FB01
:102D80000746E36A9E6916F0080617D000F0F0FBCC
:102D9000C31BFA2BF5D9FFF703FCACE70321132083
:102DA00001F044FD0321152001F040FDDAE7032185
:102DB000142001F03BFD03211620F5E79A6942F04B
:102DC00001029A6100F0D4FB0746E36A9A69D007D2
:102DD00005D400F0CDFBC31BFA2BF6D9DBE79A69CB
:102DE000002704F5825B42F002020BF1100B9A619E
:102DF000E36A5F65FFF7D4FB686CFFF799FA20225E
:102E000000216846FEF766FF02A8FFF7FFFD6A464D
:102E10000BEB06030DF1180E069794460833BCE839
:102E20000300F44543F8080C43F8041C6246F4D14F
:102E3000DCF8000020361860B6F5806F9CF804209E
:102E40001A71DCD1002304F5A252514620461A32F1
:102E500085F8503485F85334FFF7A0FE074690B943
:102E6000E26A936923F00103936100F081FB054658
:102E7000E36A9B69D9077FF53EAF00F079FB431BFE
:102E8000FA2BF5D937E795F85F6495F85E2436029A
:102E9000C5F86CA4E36A46EA426695F860241643D6
:102EA000B5F85C2446EA0246DE61B8F1000F29D08D
:102EB00004F5A352414620460232FFF76FFE90B957
:102EC000E26A936923F00103936100F051FB054628
:102ED000E36A9B69DA077FF50EAF00F049FB431BFD
:102EE000FA2BF5D907E795F8683495F867141B01B4
:102EF000C5F87084E26A43EA0123B5F8641443EA32
:102F00000143D360E36A00262046C3F8BC60FFF7A4
:102F1000AFFE85F859646FF04042E36A1A65184ABB
:102F2000E36A5A654FF00222E36A9A654FF0FF3276
:102F3000E36AC3F8E0200322E36A9145DA653FF4CF
:102F4000DBAEE26A936923F00103936100F010FBAA
:102F50000646E36A9B69DB0705D500F009FB831B86
:102F6000FA2BF6D9C7E6012385F85234C4E600BF30
:102F70002063002028630020004402582C790008B8
:102F8000550200022DE9F04F054689B0904699465A
:102F9000002741F2680A00F58056EB6AD3F8D83072
:102FA000FB40D8074AD505EB47124FEA471B52446E
:102FB0001379190742D4D6F880340133C6F8803427
:102FC00013799A0605EB0B0248BFD6F8A834524491
:102FD00044BF0133C6F8A834137943F008031371D2
:102FE000DB0723D596F8533403B305F582546846BE
:102FF000FFF712FD03AB18345C4404F1080C2068A1
:10300000083454F8041C1A46644503C21346F6D12A
:103010002068694610602846A2889A800123ADF88E
:1030200008302B68CDE90089DB6B9847D6F854341B
:1030300023B1D6F89C340133C6F89C340137202FD5
:10304000ABD109B0BDE8F08F2DE9F04F0F468DB040
:10305000044600F08FFA82468946002F5BD1E36A6E
:10306000D3F8A02012F4FE0F03D100200DB0BDE86C
:10307000F08FD3F8A420920141BF04F58051D1F81C
:1030800094240132C1F89424D3F8A4205606ECD03D
:10309000D3F8A450E669C5F305254823E8464FF068
:1030A000000B03FB05664046FFF7B0FC3268510099
:1030B0004ABF22F06043C2F38A4343F000439200C8
:1030C00048BF43F080430093736813F400131BBFA1
:1030D000012304F580528DF80D308DF80D301EBFA0
:1030E000D2F8AC340133C2F8AC34F38803F00F03E8
:1030F0008DF80C309DF80C0000F096FA5FFA8BF317
:10310000984225D9F2180CA90BF1010B127A0B4445
:1031100003F82C2CEEE7012FA7D1E36AD3F8B020F7
:1031200012F4FE0FA1D0D3F8B420950141BF04F5ED
:103130008051D1F894240132C1F89424D3F8B420FA
:10314000500692D0D3F8B450266AC5F30525A4E7FB
:10315000EFB9E36AC3F8A85004A807ADFFF75CFC19
:1031600098E80F0007C52B800023204604A9ADF87E
:103170001830236804F58054DB6BCDE904A9984727
:1031800058B1D4F88C340133C4F88C346EE7012F75
:10319000E2D1E36AC3F8B850DEE7D4F890340120F6
:1031A0000133C4F8903461E7F8B505460F4600F5E1
:1031B0008054012639462846FFF746FF10B184F8AF
:1031C0005364F7E7D4F8543423B1D4F89C34013372
:1031D000C4F89C34F8BD0000C36AF0B51A6C12F450
:1031E0007F0F2BD01B6C00F5805441F268054FF027
:1031F000010CC4F8A0340023471900EB43125E0110
:103200002A44117911F0020F15D0490713D4B95986
:10321000C66A0CFA01F1D6F8CCE011EA0E0F0AD01A
:10322000C6F8D410117941F004011171D4F8882442
:103230000132C4F888240133202BDED1F0BD000018
:103240002B4B70B51E561B5C012B30D8294D2A4ADA
:1032500055F8233052F8264013B349B3236D9A052D
:1032600010D54FF40073236500F084F950EA010291
:103270000B4602D0013861F10003024655F82600E2
:10328000FFF780FE236D9B012CD54FF0007255F89F
:103290002630226503F58053012283F8592421E06A
:1032A00001232365102323654FF48053236570BDEC
:1032B000236DDA0702D4236D5B0706D505230021B1
:1032C00055F826002365FFF76FFF236DD80602D45B
:1032D000236D590606D55023012155F82600236594
:1032E000FFF762FF55F82600BDE87040FFF774BF96
:1032F00030790008206300203479000808B5FFF712
:1033000049F9FFF769FFBDE80840FFF749B9000038
:10331000C36AD3F8C00010F07C5005D0D3F8C400C5
:1033200080F40010C0F340507047000000F580505A
:1033300008B5FFF72FF9406CFFF70CF8FFF730F9ED
:1033400043090CBF0120002008BD000000F5805398
:1033500093F8592462B1C16A8A6922F001028A6134
:10336000D3F898240132C3F89824002283F8592412
:10337000704700002DE9F74300F58251984600257B
:10338000FFF708F9103141F2680E4FF0010900F51E
:10339000805C00EB4514744423795E071CD4DB0683
:1033A0001AD58E69C36A09FA06F6D3F8CC703E4284
:1033B00012D04F6801970F689742019F77EB08077B
:1033C0000AD2C3F8D460237943F004032371DCF8F4
:1033D00084340133CCF8843401352031202DD8D108
:1033E00003B0BDE8F043FFF7DBB80000F8B51E46B8
:1033F00000230F46054613701446FFF797FF80F031
:10340000010038701EB12846FFF782FF2070F8BD1A
:103410002DE9F04F85B099460D468046164691F845
:1034200000B0DDE90EA302931378019300F0A2F837
:103430002B7804460F4613B93378002B42D022462E
:103440003B464046FFF796FFFFF758FFFFF77EFF2A
:103450004B4632462946FFF7C9FF2B7833B1BBF103
:10346000000F03D0012005B0BDE8F08F337813B111
:10347000019B002BF6D108F5805303935445029B22
:1034800077EB03031ED2039BD3F85404D0B1036837
:10349000AAEB0401DB6889B298474B4632462946BD
:1034A0004046FFF7A3FF2B7813B1BBF1000FD9D132
:1034B000337813B1019B002BD4D100F05BF80446A4
:1034C0000F46DBE70020CEE7002108B50846FFF7EE
:1034D000B7FEBDE8084001F06DB8000008B5012155
:1034E0000020FFF7ADFEBDE8084001F063B8000022
:1034F00008B500210120FFF7A3FEBDE8084001F058
:1035000059B80000012108B50846FFF799FEBDE84B
:10351000084001F04FB8000000B59BB0EFF30981FF
:1035200068226846FEF7B0FBEFF30583014B9B6B07
:10353000FEE700BF00ED00E008B5FFF7EDFF00007B
:1035400000B59BB0EFF3098168226846FEF79CFB4B
:10355000EFF30583014B5B6BFEE700BF00ED00E07E
:10356000FEE700000FB408B5029802F025F8FEE768
:1035700002F0CCBC02F0A4BC13B56C46031D84E879
:10358000060094E8030083E80500012002B010BDA6
:1035900073B58568019155B11B885B0707D4D0E9E5
:1035A00000369B6B9847019AC1B23046A84701206C
:1035B00002B070BDF0B5866889B005460C465EB1B4
:1035C000BDF838305B070AD4D0E900379B6B9847C9
:1035D0002246C1B23846B047012009B0F0BD0022F2
:1035E000002301F10806CDE9002300230A46ADF8C7
:1035F000083003AB1068083252F8041C1C46B24273
:1036000003C42346F6D1106820609288A280FFF799
:10361000B1FF0423ADF808302B68CDE90001DB6B66
:10362000694628469847D7E7082817D909280CD0B3
:103630000A280CD00B280CD00C280CD00D280CD04C
:103640000E2814BF4020302070470C2070471020F7
:1036500070471420704718207047202070470000E2
:103660002DE9F041456A15B94162BDE8F0814B682A
:10367000AC4623F06047C3F38A464FEAD37EC3F3D8
:10368000807816EA230638BF3E462B465A68BEEBC2
:10369000D27F22F060440AD0002A18DAA40CB44287
:1036A00017D19D420FD10D60DEE71346EEE7A7422A
:1036B00007D102F08044C2F3807242450BD054B16E
:1036C000EFE708D2EDE7CCF800100B60CDE7B4428D
:1036D00001D0B442E5D81A689C46002AE5D11960A9
:1036E000C3E700002DE9F047089D01F0070400EB57
:1036F000D1004FF47F494FEAD508224405F0070571
:10370000944201D1BDE8F08704F0070705F0070AED
:10371000111B08EBD50E57453E4613F80EC038BFB7
:103720005646C6F108068E4228BF0E46E108415CA7
:1037300034443544B94029FA06F721FA0AF1FFB2B8
:103740008CEA010147FA0AF739408CEA010C03F8C8
:103750000EC0D5E780EA0120082341F2210201B220
:10376000013B4000002980B2B8BF504013F0FF0376
:10377000F5D1704738B50C468D18A54200D138BD3B
:1037800014F8011BFFF7E6FFF7E7000042684AB1B3
:10379000136881894360438901339BB29942438115
:1037A00038BF83811046704770B588B00446202228
:1037B0000D4668460021FEF78DFA20460495FFF776
:1037C000E5FF024660B16B46054608AE1C4608356B
:1037D00003CCB44245F8080C45F8041C2346F5D147
:1037E000104608B070BD0000082817D909280CD071
:1037F0000A280CD00B280CD00C280CD00D280CD08B
:103800000E2814BF4020302070470C207047102035
:103810007047142070471820704720207047000020
:10382000082817D90C280CD910280CD914280CD921
:1038300018280CD920280CD930288CBF0F200E2036
:103840007047092070470A2070470B2070470C20F2
:1038500070470D20704700002DE9F843078C04469F
:10386000072F1ED900254FF6FF73D0E90298C5F146
:103870002006A5F1200029FA05F1083508FA06F618
:1038800028FA00F0314301431846C9B2FFF762FF3E
:10389000402D0346EBD13A46E169BDE8F843FFF716
:1038A00069BF4FF6FF70BDE8F883000010B54B68A4
:1038B00023B9CA8A63F30902CA8210BD04691A686F
:1038C0001C600361C38A013BC3824A60EFE70000CA
:1038D0002DE9F84F1D46CB8A0F468146C3F30901F7
:1038E000924605290B4630D00020AAB207F11A04EF
:1038F0009EB21FFA80F8042E0FD8904503F1010301
:1039000006D30A44FB8A62F309030120FB821AE012
:103910001AF800600130E654EAE79045F1D2A1F1CF
:10392000050B1C237C68BBFBF3F203FB12BB1FFAE5
:103930008BF6002C45D14846FFF728FF044638B9DE
:1039400078606FF00200BDE8F88F4FF00008E6E7FE
:10395000002606607860ADB24FF0000B454510D9E7
:103960000AEB0803221D13F8011B08F10108915509
:10397000B1B21FFA88F81B292BD0454506F1010684
:10398000F1D8FB8AC3F30902154465F30903BCE7C8
:1039900001321C4692B22368002BF9D16B1F0B44F5
:1039A0001C21B3FBF1F301339BB29A42D3D2BBF19A
:1039B000000FD0D14846FFF7E9FE20B9C4F800B0A7
:1039C000BFE70122E7E7C0F800B05E46206004468A
:1039D000C1E74545D5D94846FFF7D8FE08B920606C
:1039E000AFE7C0F800B0002620600446B6E700004C
:1039F0002DE9F04F1C46074688462DED028B83B01B
:103A00005B690192002B00F09A80238C2BB1E26954
:103A1000002A00F09480072B35D807F10C00FFF73F
:103A2000B5FE054638B96FF00205284603B0BDEC77
:103A3000028BBDE8F08F14220021FEF74BF9228C97
:103A4000E16905F10800FEF71FF9208C48F00041FC
:103A5000013080B2FFF7E4FEFFF7C6FE013880B206
:103A600020840130287438466369228C1B782A44EC
:103A700003F01F0363F03F03137269602946FFF7E9
:103A8000EFFD0125D1E74FF0000900F10C034FF0E5
:103A9000800A4E464D4608EE103A18EE100AFFF71F
:103AA00075FE83460028BED014220021FEF712F9CD
:103AB000002E3AD1019B0222ABF808300BF1080E20
:103AC0001FFA82FC218C0CF10100BCF1060F80B2C0
:103AD00001D88E422BD3FFF7A3FE8E4208BF4FF0D2
:103AE000400AFFF781FE62690138013512781BFA3E
:103AF00080F1013002F01F022DB242EA491289F032
:103B000001094AEA020A48F0004281F808A0594631
:103B10008BF810003846CBF804204FF0000AFFF76E
:103B20009FFD238CB342B8D17FE70022C6E7E1694D
:103B3000895D01360EF80210B6B20132C0E76FF0AF
:103B4000010572E7F8B515460E46302200210446FD
:103B50001F46FEF7BFF8069BB5F5001FA760636020
:103B600004F11000079B34BF6A094FF6FF72E6614B
:103B7000A362002397B29A4206D800230360A7826B
:103B8000E3822383E360F8BD0660013330462036CC
:103B9000F1E7000003781BB94BB2002BC8BF0170DE
:103BA0007047000000787047F8B50C46C9690746B1
:103BB00011B9238C002B37D1257E1F2D34D83878AE
:103BC00028BB228C072A2CD8268A36F003032BD157
:103BD0004FF6FF70FFF7CEFD20F0010031024FF6E7
:103BE000FF72400441EA0561400C41EA402523464A
:103BF00029463846FFF7FCFE002807DD6269137886
:103C00000133DBB21F2B88BF00231370F8BD218A5C
:103C10002D0645EA012505432046FFF71DFE024615
:103C2000E5E76FF00300F1E76FF00100EEE7000059
:103C300070B58AB0044616460021282268461D4603
:103C4000FEF748F8BDF8383069462046ADF8103028
:103C50000F9B05939DF840308DF81830119B07930A
:103C6000BDF84830CDE90265ADF82030FFF79CFF84
:103C70000AB070BD2DE9F041D36905460C461646E1
:103C80000BB9138C5BBB377E1F2F28D895F80080AB
:103C9000B8F1000F26D03046FFF7DEFD3378210261
:103CA0000246284641EAC331338A41EA080141EA23
:103CB000076141EA0341334641F08001FFF798FE76
:103CC00000280ADD3378012B07D17269137801339C
:103CD000DBB21F2B88BF00231370BDE8F0816FF0AB
:103CE0000100FAE76FF00300F7E70000F0B58BB0D2
:103CF00004460D4617460021282268461E46FDF759
:103D0000E9FF9DF84C30294620465A1E5342534144
:103D10006A468DF800309DF84030ADF81030119BA8
:103D200005939DF848308DF81830149B0793BDF823
:103D30005430CDE90276ADF82030FFF79BFF0BB091
:103D4000F0BD0000406A00B104307047436A1A6851
:103D5000426202691A600361C38A013BC3827047F1
:103D60002DE9F041D0F8208014461D46184E4146FA
:103D7000002709B9BDE8F081D1E90223A21A65EB59
:103D80000303964277EB03031ED2036A8B420DD1E5
:103D9000FFF78CFD036A1B68036203690B60C38A2B
:103DA0000161013B016AC3828846E2E7FFF77EFDBD
:103DB0000B68C8F8003003690B60C38A0161013BDE
:103DC000C382D8F80010D4E788460968D1E700BF5D
:103DD00080841E002DE9F04F8BB00D4614469B46A3
:103DE000DDF850908046002800F01881B9F1000FEE
:103DF00000F01481531E3F2B00F21081012A03D1E1
:103E0000BBF1000F40F00A810023CDE90833B8F878
:103E10001430B5EBC30F4FEAC30703D300200BB038
:103E2000BDE8F08F2B199F42D8F80C3036BF7F1BAE
:103E30002746FFB21BB9D8F81030002B7AD0272DB7
:103E40004DD8C5F1280600232946B742009308AB98
:103E5000D8F808002CBFF6B23E46A7EB060A354458
:103E600032465FFA8AFAFFF73DFCB8F81430282191
:103E700003F10053053BDB000493D8F80C300393A7
:103E8000039B13B1BAF1000F2CD1D8F8100040B148
:103E9000BAF1000F05D008AB5246691A0096FFF739
:103EA00021FC38B2002FB9D066070AD00AAB6242B3
:103EB00003EBD40102F0070211F8083C134101F8AA
:103EC000083C082C3DD9102C40F2B580202C40F243
:103ED000B780BBF1000F00F09C80082335E0BA46A4
:103EE0000026C2E7049BE02B28BFE02306930B4487
:103EF000AB42059315D95A1B0398691A009692454F
:103F000008AB00F1040034BF5246D2B20792FFF76B
:103F1000E9FB079A1644AAEB020A1544F6B25FFAC7
:103F20008AFA049B069A05999B1A0493039B1B68C3
:103F30000393A5E700933A4608AB2946D8F8080052
:103F4000ADE7BBF1000F13D00123B4EBC30F6BD06F
:103F5000082C12D89DF82030621E23FA02F2D507F1
:103F600006D54FF0FF3202FA04F423438DF82030D7
:103F70009DF8203089F8003051E7102C12D8BDF898
:103F80002030621E23FA02F2D10706D54FF0FF322D
:103F900002FA04F42343ADF82030BDF82030A9F82C
:103FA00000303CE7202C0FD80899631E21FA03F358
:103FB000DA0705D54FF0FF3202FA04F40C430894F7
:103FC000089BC9F800302AE7402C2AD0611EC4F1B2
:103FD0002102A4F12103DDE9086526FA01F105FAC1
:103FE00002F225FA03F311431943CB0711D501223D
:103FF000A4F12003C4F1200102FA03F322FA01F133
:10400000A2400B43524263EB430332432B43CDE9BF
:104010000823DDE90823C9E9002300E76FF0010068
:10402000FDE66FF00800FAE6082CA1D9102CB4D9EF
:10403000202CEED8C4E7BBF1000FAED0022384E7FA
:10404000BBF1000FBCD004237FE70000012A30B58C
:10405000144638BF012485B00025402C28BF4024D9
:10406000012ACDE9025518D81B788DF8083063076E
:104070000AD004AB624203EBD40502F0070215F844
:10408000083C934005F8083C034600912246002175
:1040900002A8FFF727FB05B030BD082AE4D9102A93
:1040A00003D81B88ADF80830E1E7202A95BF1B68CC
:1040B000D3E900230293CDE90223D8E710B5CB68FA
:1040C0001BB98B600B618B8210BD04691A681C6080
:1040D0000361C38A013BC382CA60F0E703064CBF99
:1040E000C0F3C0300220704708B50246FFF7F6FF64
:1040F000022806D15306C2F30F2001D100F00300BD
:1041000008BDC2F30740FBE72DE9F04F93B004462A
:104110000D46CDE903230A681046FFF7DFFF0228AA
:10412000824614BFC2F306260026002A80F2F381DD
:1041300012F0C04940F0EF81097B002900F0EB81CB
:10414000022803D02378B34240F0E881C2F304632D
:1041500010462944069302F07F030593FFF7C4FF3E
:10416000059B002283464FEA8348002348EA0A4819
:1041700048EA4668CE78CDE90823F30948EA000802
:10418000029368D0059B024608A920460093534637
:104190006768B847002800F0C481276A4FB94146D4
:1041A00004F10C00FFF700FB074690B96FF0020026
:1041B00055E03B6998450DD03F68002FF9D1414645
:1041C00004F10C00FFF7F0FA07460028EED0236A4E
:1041D0003B60276297F817C006F01F08CCF3840CE9
:1041E000ACEB0800A8EB0C031FFA80FE0028B8BF58
:1041F0000EF120001FFA83FEB8BF00B2002B079318
:10420000B8BF0EF12003D7E90221BCBF1BB2079350
:1042100052EA010338D0039B4FF0000CDFF820E393
:104220009A1A049B63EB010196457CEB01032BD3A7
:104230006B7B97F81AE0734519D1029B002B78D05D
:10424000012821DC7868F8B9DFF8F0C2944570EBFA
:10425000010316D337E0276A27B96FF00C0013B0BB
:10426000BDE8F08F3B699845B4D03F68F4E7B348A8
:1042700090427CEB010301D30020F0E7029B002B6E
:10428000FAD0079B0F2B17DCFA7DB3003946204686
:1042900002F0030203F07C031343FB75FFF706FBF8
:1042A0006B7BBB76029B3BB9FB7DC3F3840201327F
:1042B00062F38603FB75D0E76A7BBB7E9A42DBD153
:1042C000029B002B35D0B309022B32D0039B142262
:1042D00000210DA8BB60049BFB60FDF7FBFC039B6A
:1042E0000AA920460A93049BADF83EB00B932B1D00
:1042F0008DF840A00C932B7B8DF84180013BDBB205
:10430000ADF83C30069B8DF84230059B8DF843306C
:1043100094F82C3083F001038DF84430A36898475B
:10432000FB7DC3F38403013303F01F039B02FB8275
:10433000A2E7FB7DC6F34012B2EBD31F40F0F4803E
:10434000C3F38403434540F0F280029AB6092B7B05
:10435000002A4DD0F2075DD4032B40F2EB80039B83
:10436000AE1D394604F10C00BB603246049BFB6075
:104370002B7B033BDBB2FFF7ABFA00280CDA3946A4
:104380002046FFF793FAFB7DC3F38403013303F068
:104390001F039B02FB8209E7AB88DDE908843B83AE
:1043A0004FF6FF73C9F12000A9F1200228FA09F1A4
:1043B00009F1080904FA00F024FA02F20143184650
:1043C0001143C9B2FFF7C6F9B9F1400F0346E9D16D
:1043D000B88231462A7B033AD2B2FFF7CBF9FB7D94
:1043E000B882DA43C2F3C01262F3C713FB7543E726
:1043F00086B92E1D013B394604F10C00DBB2324672
:10440000FFF766FA0028BADB2A7B3146B88A013A00
:10441000D2B2E2E7F98A013BC1F30901DAB2042919
:104420005BD8281D002307F11B069A4208D910F813
:1044300001CB013306F801C00131DBB20529F4D10B
:10444000039993420A9138BF043304992CBF002387
:1044500055FA83F30B9107F11B010C9179680E93C8
:104460000D91291DFB8AADF83EB0C3F309038DF809
:1044700040A08DF841801A44069B8DF84230059B80
:10448000ADF83C208DF8433094F82C3083F00103D4
:104490008DF844300023B88A7B602A7B013AFFF70D
:1044A00069F93B8BB882834203D1A3680AA92046ED
:1044B000984720460AA9FFF701FEFB7DBA8AC3F39D
:1044C0008403013303F01F039B02FB823B8B9A4260
:1044D0000CBF00206FF01000C1E67B68002BAFD04E
:1044E000052001E01C3033461E68002EFAD1091A5F
:1044F0002E1D081D184401EB090C5FFA89F3BCF16D
:104500001B0F9DD89A429BD916F8013B09F101096E
:1045100000F8013BEFE76FF00900A0E66FF00A003A
:104520009DE66FF00B009AE66FF00D0097E66FF0D6
:104530000E0094E66FF00F0091E600BF40420F00BE
:1045400080841E00EFF30983054968334A6B22F02B
:1045500001024A6383F30988002383F311887047BB
:1045600000EF00E0302080F3118862B60D4B0E4A58
:10457000D96821F4E0610904090C0A430B49DA60A7
:10458000D3F8FC2042F08072C3F8FC20084AC2F83D
:10459000B01F116841F0010111602022DA7783F821
:1045A0002200704700ED00E00003FA0555CEACC5CF
:1045B000001000E0302310B583F311880E4B5B68C8
:1045C00013F4006314D0F1EE103AEFF309844FF0C6
:1045D0008073683CE361094BDB6B236684F30988D5
:1045E00000F0A8FF10B1064BA36110BD054BFBE71F
:1045F00083F31188F9E700BF00ED00E000EF00E071
:104600004307000846070008026843681143016039
:1046100003B1184770470000024A136843F0C00313
:10462000136070470078004013B50E4C204600F030
:10463000A7FA04F1140000234FF400720A49009411
:1046400000F064F9094B4FF40072094904F1380095
:10465000009400F0DDF9074A074BC4E9172302B0C4
:1046600010BD00BF34630020A0630020194600087D
:10467000A06500200078004000E1F505037C30B51E
:10468000244C002918BF0C46012B11D1224B984213
:104690000ED1224BD3F8E82042F08042C3F8E82044
:1046A000D3F8102142F08042C3F81021D3F8103122
:1046B0002268036EC16D03EB52038466B3FBF2F311
:1046C0006268150442BF23F0070503F0070343EABD
:1046D0004503CB60A36843F040034B60E36843F0BD
:1046E00001038B6042F4967343F001030B604FF0BB
:1046F000FF330B62510505D512F0102205D0B2F13F
:10470000805F04D080F8643030BD7F23FAE73F2318
:10471000F8E700BF847900083463002000440258A1
:104720002DE9F047C66D05463768F4692107346204
:104730001AD014F0080118BF4FF48071E20748BF87
:1047400041F02001A3074FF0300348BF41F0400182
:10475000600748BF41F0800183F31188281DFFF7EF
:1047600053FF002383F31188E2050AD5302383F336
:1047700011884FF48061281DFFF746FF002383F363
:1047800011884FF030094FF0000A14F0200838D19A
:104790003B0616D54FF0300905F1380A200610D532
:1047A00089F31188504600F067F9002836DA0821AD
:1047B000281DFFF729FF27F080033360002383F3D0
:1047C0001188790614D5620612D5302383F3118837
:1047D000D5E913239A4208D12B6C33B127F0400757
:1047E0001021281DFFF710FF3760002383F3118885
:1047F000E30618D5AA6E1369ABB15069BDE8F0475E
:10480000184789F31188736A284695F8641019408F
:1048100000F0D0F98AF31188F469B6E7B06288F342
:104820001188F469BAE7BDE8F0870000090100F1DA
:104830006043012203F56143C9B283F8001300F01D
:104840001F039A4043099B0003F1604303F5614352
:10485000C3F880211A607047F8B51546826804468F
:104860000B46AA4200D28568A1692669761AB5422C
:104870000BD218462A46FDF707FAA3692B44A36119
:104880002846A3685B1BA360F8BD0CD9AF1B184674
:104890003246FDF7F9F93A46E1683044FDF7F4F99C
:1048A000E3683B44EBE718462A46FDF7EDF9E36879
:1048B000E5E7000083689342F7B50446154600D249
:1048C0008568D4E90460361AB5420BD22A46FDF752
:1048D000DBF963692B4463612846A3685B1BA36013
:1048E00003B0F0BD0DD93246AF1B0191FDF7CCF9F5
:1048F00001993A46E0683144FDF7C6F9E3683B4464
:10490000E9E72A46FDF7C0F9E368E4E710B50A4491
:104910000024C361029B8460C16002610362C0E93C
:104920000000C0E9051110BD08B5D0E90532934279
:1049300001D1826882B98268013282605A1C426168
:1049400019700021D0E904329A4224BFC368436140
:1049500000F0C2FE002008BD4FF0FF30FBE7000072
:1049600070B5302304460E4683F31188A568A5B1BF
:10497000A368A269013BA360531CA3611578226957
:10498000934224BFE368A361E3690BB120469847D3
:10499000002383F31188284607E03146204600F0C3
:1049A0008BFE0028E2DA85F3118870BD2DE9F74F00
:1049B00004460E4617469846D0F81C904FF0300A31
:1049C0008AF311884FF0000B154665B12A4631462F
:1049D0002046FFF741FF034660B94146204600F0FC
:1049E0006BFE0028F1D0002383F31188781B03B0FD
:1049F000BDE8F08FB9F1000F03D001902046C84701
:104A0000019B8BF31188ED1A1E448AF31188DCE7B1
:104A1000C160C361009B82600362C0E9051111445B
:104A2000C0E9000001617047F8B504460D4616461E
:104A3000302383F31188A768A7B1A368013BA36063
:104A400063695A1C62611D70D4E904329A4224BF22
:104A5000E3686361E3690BB120469847002080F367
:104A6000118807E03146204600F026FE0028E2DAF1
:104A700087F31188F8BD0000D0E9052310B59A42EC
:104A800001D182687AB982680021013282605A1CA1
:104A900082611C7803699A4224BFC368836100F075
:104AA0001BFE204610BD4FF0FF30FBE72DE9F74F0E
:104AB00004460E4617469846D0F81C904FF0300A30
:104AC0008AF311884FF0000B154665B12A4631462E
:104AD0002046FFF7EFFE034660B94146204600F04E
:104AE000EBFD0028F1D0002383F31188781B03B07D
:104AF000BDE8F08FB9F1000F03D001902046C84700
:104B0000019B8BF31188ED1A1E448AF31188DCE7B0
:104B1000026843681143016003B118477047000001
:104B20001430FFF743BF00004FF0FF331430FFF79E
:104B30003DBF00003830FFF7B9BF00004FF0FF3332
:104B40003830FFF7B3BF00001430FFF709BF000093
:104B50004FF0FF311430FFF703BF00003830FFF78C
:104B600063BF00004FF0FF323830FFF75DBF000039
:104B7000012914BF6FF0130000207047FFF754BDE8
:104B8000044B036000234360C0E902330123037434
:104B9000704700BF9C79000810B53023044683F3AA
:104BA0001188FFF76BFD02230020237480F3118826
:104BB00010BD000038B5C36904460D461BB9042179
:104BC0000844FFF7A5FF294604F11400FFF7ACFEE7
:104BD000002806DA201D4FF40061BDE83840FFF7D9
:104BE00097BF38BD026843681143016003B118479D
:104BF0007047000013B5406B00F58054D4F8A4381A
:104C00001A681178042914D1017C022911D119796B
:104C1000012312898B4013420BD101A94C3002F0C1
:104C200017F9D4F8A4480246019B2179206800F0C6
:104C3000DFF902B010BD0000143002F099B8000096
:104C40004FF0FF33143002F093B800004C3002F004
:104C50006BB900004FF0FF334C3002F065B9000033
:104C6000143002F067B800004FF0FF31143002F04A
:104C700061B800004C3002F037B900004FF0FF324D
:104C80004C3002F031B900000020704710B500F53B
:104C90008054D4F8A4381A681178042917D1017CFB
:104CA000022914D15979012352898B4013420ED124
:104CB000143001F0F9FF024648B1D4F8A4484FF48B
:104CC000407361792068BDE8104000F07FB910BDE5
:104CD000406BFFF7DBBF0000704700007FB5124B51
:104CE00001250426044603600023057400F18402B4
:104CF00043602946C0E902330C4B02901430019303
:104D00004FF44073009601F0ABFF094B04F6944258
:104D1000294604F14C000294CDE900634FF440733E
:104D200002F072F804B070BDC4790008D14C0008DC
:104D3000F54B00080A68302383F311880B790B3395
:104D400042F823004B79133342F823008B7913B1D7
:104D50000B3342F8230000F58053C3F8A418022354
:104D60000374002080F311887047000038B5037F7A
:104D7000044613B190F85430ABB90125201D02212F
:104D8000FFF730FF04F114006FF00101257700F008
:104D9000AFFC04F14C0084F854506FF00101BDE801
:104DA000384000F0A5BC38BD10B5012104460430E0
:104DB000FFF718FF0023237784F8543010BD00005C
:104DC00038B504460025143001F062FF04F14C00B0
:104DD000257702F031F8201D84F854500121FFF7A7
:104DE00001FF2046BDE83840FFF750BF90F8803003
:104DF00003F06003202B06D190F881200023212AA4
:104E000003D81F2A06D800207047222AFBD1C0E908
:104E10001D3303E0034A426707228267C36701200C
:104E2000704700BF3C22002037B500F58055D5F80B
:104E3000A4381A68117804291AD1017C022917D1E3
:104E40001979012312898B40134211D100F14C04CE
:104E5000204602F0B1F858B101A9204601F0F8FF50
:104E6000D5F8A4480246019B2179206800F0C0F8DB
:104E700003B030BD01F10B03F0B550F8236085B0ED
:104E800004460D46FEB1302383F3118804EB8507F9
:104E9000301D0821FFF7A6FEFB6806F14C005B6998
:104EA0001B681BB1019001F0E1FF019803A901F01B
:104EB000CFFF024648B1039B2946204600F098F8F0
:104EC000002383F3118805B0F0BDFB685A691268AE
:104ED000002AF5D01B8A013B1340F1D104F1800276
:104EE000EAE70000133138B550F82140ECB1302327
:104EF00083F3118804F58053D3F8A42813685279FA
:104F000003EB8203DB689B695D6845B1042160188F
:104F1000FFF768FE294604F1140001F0CFFE204699
:104F2000FFF7B4FE002383F3118838BD70470000FB
:104F300001F09CB901234022002110B5044600F87D
:104F4000303BFCF7C7FE0023C4E9013310BD00006D
:104F500010B53023044683F31188242241600021D8
:104F60000C30FCF7B7FE204601F0A2F90223002026
:104F7000237080F3118810BD70B500EB81030546E6
:104F800050690E461446DA6018B110220021FCF771
:104F9000A1FEA06918B110220021FCF79BFE31464A
:104FA0002846BDE8704001F089BA000083682022DD
:104FB000002103F0011310B5044683601030FCF7A4
:104FC00089FE2046BDE8104001F004BBF0B4012585
:104FD00000EB810447898D40E4683D43A469458125
:104FE00023600023A2606360F0BC01F021BB0000DD
:104FF000F0B4012500EB810407898D40E4683D434E
:105000006469058123600023A2606360F0BC01F045
:1050100097BB000070B502230025044624220370CC
:105020002946C0F888500C3040F8045CFCF752FE6A
:10503000204684F8705001F0D5F963681B6823B1ED
:1050400029462046BDE87040184770BD0378052BFF
:1050500010B504460AD080F88C30052303704368ED
:105060001B680BB1042198470023A36010BD00000A
:105070000178052906D190F88C20436802701B68DE
:1050800003B118477047000070B590F870300446BF
:1050900013B1002380F8703004F18002204601F043
:1050A000BDFA63689B68B3B994F8803013F060056B
:1050B00035D00021204601F0AFFD0021204601F04F
:1050C0009FFD63681B6813B106212046984706239D
:1050D00084F8703070BD204698470028E4D0B4F8BA
:1050E0008630A26F9A4288BFA36794F98030A56F7B
:1050F000002B4FF0300380F20381002D00F0F2808E
:10510000092284F8702083F3118800212046D4E915
:105110001D23FFF76DFF002383F31188DAE794F86E
:10512000812003F07F0343EA022340F202329342DC
:1051300000F0C58021D8B3F5807F48D00DD8012B71
:105140003FD0022B00F09380002BB2D104F18802F3
:1051500062670222A267E367C1E7B3F5817F00F0CF
:105160009B80B3F5407FA4D194F88230012BA0D16D
:10517000B4F8883043F0020332E0B3F5006F4DD04D
:1051800017D8B3F5A06F31D0A3F5C063012B90D829
:105190006368204694F882205E6894F88310B4F81F
:1051A0008430B047002884D0436863670368A367EE
:1051B0001AE0B3F5106F36D040F6024293427FF406
:1051C00078AF5C4B63670223A3670023C3E794F8BF
:1051D0008230012B7FF46DAFB4F8883023F00203E6
:1051E000A4F88830C4E91D55E56778E7B4F8803045
:1051F000B3F5A06F0ED194F88230204684F88A303F
:1052000001F04EF963681B6813B1012120469847ED
:10521000032323700023C4E91D339CE704F18B03AF
:1052200063670123C3E72378042B10D1302383F372
:1052300011882046FFF7BAFE85F3118803216368C1
:1052400084F88B5021701B680BB12046984794F866
:105250008230002BDED084F88B3004232370636807
:105260001B68002BD6D0022120469847D2E794F83D
:10527000843020461D0603F00F010AD501F0C0F965
:10528000012804D002287FF414AF2B4B9AE72B4B54
:1052900098E701F0A7F9F3E794F88230002B7FF448
:1052A00008AF94F8843013F00F01B3D01A062046EB
:1052B00002D501F0C9FCADE701F0BAFCAAE794F809
:1052C0008230002B7FF4F5AE94F8843013F00F0198
:1052D000A0D01B06204602D501F09EFC9AE701F003
:1052E0008FFC97E7142284F8702083F311882B46F3
:1052F0002A4629462046FFF769FE85F31188E9E62C
:105300005DB1152284F8702083F3118800212046B6
:10531000D4E91D23FFF75AFEFDE60B2284F8702026
:1053200083F311882B462A4629462046FFF760FE64
:10533000E3E700BFF4790008EC790008F079000891
:1053400038B590F870300446002B3ED0063BDAB2F8
:105350000F2A34D80F2B32D8DFE803F03731310869
:10536000223231313131313131313737856FB0F857
:1053700086309D4214D2C3681B8AB5FBF3F203FB4F
:1053800012556DB9302383F311882B462A462946DE
:10539000FFF72EFE85F311880A2384F870300EE0A3
:1053A000142384F87030302383F3118800232046BF
:1053B0001A461946FFF70AFE002383F3118838BD09
:1053C000C36F03B198470023E7E70021204601F0AF
:1053D00023FC0021204601F013FC63681B6813B115
:1053E0000621204698470623D7E7000010B590F81D
:1053F00070300446142B29D017D8062B05D001D8BD
:105400001BB110BD093B022BFBD80021204601F047
:1054100003FC0021204601F0F3FB63681B6813B115
:10542000062120469847062319E0152BE9D10B23C6
:1054300080F87030302383F3118800231A46194610
:10544000FFF7D6FD002383F31188DAE7C3689B6971
:105450005B68002BD5D1C36F03B19847002384F854
:105460007030CEE700238268037503691B68996872
:105470009142FBD25A6803604260106058607047E6
:1054800000238268037503691B6899689142FBD801
:105490005A680360426010605860704708B508465B
:1054A000302383F311880B7D032B05D0042B0DD003
:1054B0002BB983F3118808BD8B6900221A604FF065
:1054C000FF338361FFF7CEFF0023F2E7D1E900321B
:1054D00013605A60F3E70000FFF7C4BF054BD968BB
:1054E00008751868026853601A600122D860027556
:1054F000FBF712B9A06700200C4B30B5DD684B1CE0
:1055000087B004460FD02B46094A684600F084F95C
:105510002046FFF7E3FF009B13B1684600F086F9D1
:10552000A86907B030BDFFF7D9FFF9E7A0670020F1
:105530009D540008044B1A68DB6890689B68984289
:1055400094BF002001207047A0670020084B10B5D1
:105550001C68D868226853601A600122DC602275DA
:10556000FFF78EFF01462046BDE81040FBF7D4B898
:10557000A0670020044B1A68DB6892689B689A4217
:1055800001D9FFF7E3BF7047A067002038B5074C8B
:1055900001230025064907482370656001F04AFD94
:1055A0000223237085F3118838BD00BF086A0020EC
:1055B000FC790008A067002008B572B6044B186596
:1055C00000F06CFC00F03EFD024B03221A70FEE777
:1055D000A0670020086A002000F05EB9EFF3118098
:1055E00020B9EFF30583302282F311887047000061
:1055F00010B530B9EFF30584C4F3080414B180F397
:10560000118810BDFFF7B6FF84F31188F9E7000099
:10561000034A516853685B1A9842FBD8704700BF31
:10562000001000E08B600223086108468B827047FF
:105630008368A3F1840243F8142C026943F8442CD4
:10564000426943F8402C094A43F8242CC268A3F16C
:10565000200043F8182C022203F80C2C002203F837
:105660000B2C034A43F8102C704700BF3107000889
:10567000A067002008B5FFF7DBFFBDE80840FFF793
:105680002BBF0000024BDB6898610F20FFF726BF9D
:10569000A0670020302383F31188FFF7F3BF0000D9
:1056A00008B50146302383F311880820FFF724FF53
:1056B000002383F3118808BD064BDB6839B14268CB
:1056C00018605A60136043600420FFF715BF4FF065
:1056D000FF307047A06700200368984206D01A6820
:1056E0000260506018469961FFF7F6BE70470000EF
:1056F00038B504460D462068844200D138BD0368A1
:1057000023605C608561FFF7E7FEF4E7036810B58E
:105710009C68A2420CD85C688A600B604C60216077
:10572000596099688A1A9A604FF0FF33836010BD00
:10573000121B1B68ECE700000A2938BF0A2170B56C
:1057400004460D460A26601901F06CFC01F054FC79
:10575000041BA54203D8751C04462E46F3E70A2E07
:1057600004D90120BDE8704001F0A4BC70BD000068
:10577000F8B5144B0D460A2A4FF00A07D96103F118
:105780001001826038BF0A22416019691446016025
:1057900048601861A81801F035FC01F02DFC431B8E
:1057A0000646A34206D37C1C28192746354601F03D
:1057B00039FCF2E70A2F04D90120BDE8F84001F0D6
:1057C00079BCF8BDA0670020F8B506460D4601F08B
:1057D00013FC0F4A134653F8107F9F4206D12A4606
:1057E00001463046BDE8F840FFF7C2BFD169BB684B
:1057F000441A2C1928BF2C46A34202D92946FFF788
:105800009BFF224631460348BDE8F840FFF77EBFC4
:10581000A0670020B0670020C0E90323002310B474
:105820005DF8044B4361FFF7CFBF000010B5194C82
:10583000236998420DD08168D0E9003213605A6024
:105840009A680A449A60002303604FF0FF33A36113
:1058500010BD0268234643F8102F536000220260F7
:1058600022699A4203D1BDE8104001F0D5BB93688C
:1058700081680B44936001F0BFFB2269E169926883
:10588000441AA242E4D91144BDE81040091AFFF7B6
:1058900053BF00BFA06700202DE9F047DFF8BC80B0
:1058A00008F110072C4ED8F8105001F0A5FBD8F8DD
:1058B0001C40AA68031B9A423ED814444FF00009CA
:1058C000D5E90032C8F81C4013605A60C5F8009052
:1058D000D8F81030B34201D101F09EFB89F3118852
:1058E000D5E9033128469847302383F311886B6943
:1058F000002BD8D001F080FB6A69A0EB0409824636
:105900004A450DD2022001F0D5FB0022D8F8103014
:10591000B34208D151462846BDE8F047FFF728BFFB
:10592000121A2244F2E712EB09092946384638BF19
:105930004A46FFF7EBFEB5E7D8F81030B34208D07F
:105940001444C8F81C00211AA960BDE8F047FFF70D
:10595000F3BEBDE8F08700BFB0670020A06700205D
:1059600000207047FEE70000704700004FF0FF3056
:105970007047000002290CD0032904D001290748F0
:1059800018BF00207047032A05D8054800EBC20065
:105990007047044870470020704700BFD47A000861
:1059A0004C220020887A000870B59AB00546084657
:1059B000144601A900F0C2F801A8FCF783F9431CC2
:1059C0000022C6B25B001046C5E9003423700323F1
:1059D000023404F8013C01ABD1B202348E4201D84A
:1059E0001AB070BD13F8011B013204F8010C04F861
:1059F000021CF1E708B5302383F311880348FFF751
:105A000013FA002383F3118808BD00BF106A002039
:105A100090F8803003F01F02012A07D190F881200E
:105A20000B2A03D10023C0E91D3315E003F0600306
:105A3000202B08D1B0F884302BB990F88120212A8E
:105A400003D81F2A04D8FFF7D1B9222AEBD0FAE7EE
:105A5000034A426707228267C3670120704700BF7D
:105A60004322002007B5052917D8DFE801F01916F1
:105A700003191920302383F31188104A0121019062
:105A8000FFF77AFA019802210D4AFFF775FA0D48DF
:105A9000FFF796F9002383F3118803B05DF804FB48
:105AA000302383F311880748FFF760F9F2E73023CA
:105AB00083F311880348FFF777F9EBE7287A0008AA
:105AC0004C7A0008106A002038B50C4D0C4C2A4660
:105AD0000C4904F10800FFF767FF05F1CA0204F161
:105AE00010000949FFF760FF05F5CA7204F11800BC
:105AF0000649BDE83840FFF757BF00BFE8820020E5
:105B00004C220020087A0008127A00081D7A00084A
:105B100070B5044608460D46FCF7D4F8C6B22046D8
:105B2000013403780BB9184670BD32462946FCF79C
:105B3000B5F80028F3D10120F6E700002DE9F04781
:105B400005460C46FCF7BEF82B49C6B22846FFF7BF
:105B5000DFFF08B10A36F6B228492846FFF7D8FF1A
:105B600008B11036F6B2632E0BD8DFF88C80DFF860
:105B70008C90234FDFF894A02E7846B92670BDE8AC
:105B8000F08729462046BDE8F04701F073BE252E78
:105B90002ED1072241462846FCF780F870B9194BF0
:105BA000224603F1100153F8040B8B4242F8040B18
:105BB000F9D11B78073511341370DDE70822494607
:105BC0002846FCF76BF898B9A21C0F4B19780232E3
:105BD0000909C95D02F8041C13F8011B01F00F014B
:105BE0005345C95D02F8031CF0D118340835C3E7EA
:105BF000013504F8016BBFE7F47A00081D7A00084C
:105C0000FC7A00089278000800E8F11F0CE8F11F08
:105C1000BFF34F8F044B1A695107FCD1D3F8102101
:105C20005207F8D1704700BF0020005208B50D4B55
:105C30001B78ABB9FFF7ECFF0B4BDA68D10704D543
:105C40000A4A5A6002F188325A60D3F80C21D2070E
:105C500006D5064AC3F8042102F18832C3F80421AC
:105C600008BD00BF46850020002000522301674583
:105C700008B5114B1B78F3B9104B1A69510703D5BE
:105C8000DA6842F04002DA60D3F81021520705D5F5
:105C9000D3F80C2142F04002C3F80C21FFF7B8FF03
:105CA000064BDA6842F00102DA60D3F80C2142F0C8
:105CB0000102C3F80C2108BD4685002000200052D7
:105CC0000F289ABF00F58060400400207047000054
:105CD0004FF4003070470000102070470F2808B5BF
:105CE0000BD8FFF7EDFF00F500330268013204D155
:105CF00004308342F9D1012008BD0020FCE70000F8
:105D00000F2838B505463FD8FFF782FF1F4CFFF735
:105D10008DFF4FF0FF3307286361C4F814311DD89D
:105D20002361FFF775FF030243F02403E360E36898
:105D300043F08003E36023695A07FCD42846FFF749
:105D400067FFFFF7BDFF4FF4003100F057F9284619
:105D5000FFF78EFFBDE83840FFF7C0BFC4F8103131
:105D6000FFF756FFA0F108031B0243F02403C4F819
:105D70000C31D4F80C3143F08003C4F80C31D4F862
:105D800010315B07FBD4D9E7002038BD002000525A
:105D90002DE9F84F05460C46104645EA0203DE069B
:105DA00002D00020BDE8F88F20F01F00DFF8BCB063
:105DB000DFF8BCA0FFF73AFF04EB0008444503D12D
:105DC0000120FFF755FFEDE720222946204601F08C
:105DD0001FFD10B920352034F0E72B4605F12002D5
:105DE0001F68791CDDD104339A42F9D105F178435B
:105DF0001B481C4EB3F5801F1B4B38BF184603F1E0
:105E0000F80332BFD946D1461E46FFF701FF0760AF
:105E1000A5EB040C336804F11C0143F0020333606A
:105E2000231FD9F8007017F00507FAD153F8042F93
:105E30008B424CF80320F4D1BFF34F8FFFF7E8FEFD
:105E40004FF0FF332022214603602846336823F0B9
:105E50000203336001F0DCFC0028BBD03846B0E719
:105E6000142100520C200052142000521020005225
:105E70001021005210B5084C237828B11BB9FFF748
:105E8000D5FE0123237010BD002BFCD02070BDE88F
:105E90001040FFF7EDBE00BF4685002038B5054D28
:105EA00000240334696855F80C0B00F0B9F8122C83
:105EB000F7D138BD107B0008084601F0A1BC0000F6
:105EC00070B5104E82B0FFF789FB054601F094F8DB
:105ED000326803469042336037BF0B4A0A49516823
:105EE000146836BF0131D1E90041516004192846D8
:105EF00041F100010191FFF77BFB2046019902B0BF
:105F000070BD00BF488500205085002070B5124E3E
:105F100082B0FFF763FB054601F06EF83268034676
:105F20009042336037BF0D4A0C495168146836BF40
:105F30000131D1E9004151600419284641F10001C5
:105F40000191FFF755FB4FF47A7200232046019927
:105F5000FAF7CEF902B070BD4885002050850020C8
:105F60000244074BD2B210B5904200D110BD441C80
:105F700000B253F8200041F8040BE0B2F4E700BF90
:105F8000504000580E4B30B51C6F240405D41C6FD4
:105F90001C671C6F44F400441C670A4C02442368CD
:105FA000D2B243F480732360074B904200D130BDDE
:105FB000441C51F8045B00B243F82050E0B2F4E70F
:105FC00000440258004802585040005807B50122CA
:105FD00001A90020FFF7C4FF019803B05DF804FB9E
:105FE00013B50446FFF7F2FFA04205D0012201A934
:105FF00000200194FFF7C6FF02B010BD0144BFF3BB
:106000004F8F064B884204D3BFF34F8FBFF36F8F80
:106010007047C3F85C022030F4E700BF00ED00E0F9
:106020000144BFF34F8F064B884204D3BFF34F8F19
:10603000BFF36F8F7047C3F870022030F4E700BFE2
:1060400000ED00E070470000074B45F255521A6022
:1060500002225A6040F6FF729A604CF6CC421A60F7
:106060000122024B1A707047004800585C850020DE
:10607000034B1B781BB1034B4AF6AA221A607047E8
:106080005C85002000480058034B1A681AB9034A7F
:10609000D2F8D0241A60704758850020004002587A
:1060A000024B4FF48032C3F8D024704700400258AE
:1060B00008B5FFF7E9FF024B1868C0F3806008BD20
:1060C0005885002070B5BFF34F8FBFF36F8F1A4A0A
:1060D0000021C2F85012BFF34F8FBFF36F8F536987
:1060E00043F400335361BFF34F8FBFF36F8FC2F898
:1060F0008410BFF34F8FD2F8803043F6E074C3F3BF
:10610000C900C3F34E335B0103EA0406014646EAC5
:1061100081750139C2F86052F9D2203B13F1200F8A
:10612000F2D1BFF34F8F536943F480335361BFF310
:106130004F8FBFF36F8F70BD00ED00E0FEE70000F2
:10614000214B2248224A70B5904237D3214BC11EC1
:10615000DA1C121A22F003028B4238BF00220021FF
:10616000FBF7B8FD1C4A0023C2F88430BFF34F8F01
:10617000D2F8803043F6E074C3F3C900C3F34E3362
:106180005B0103EA0406014646EA81750139C2F85B
:106190006C52F9D2203B13F1200FF2D1BFF34F8F95
:1061A000BFF36F8FBFF34F8FBFF36F8F0023C2F822
:1061B0005032BFF34F8FBFF36F8F70BD53F8041B86
:1061C00040F8041BC0E700BFB07D00083087002006
:1061D000308700203087002000ED00E0074BD3F827
:1061E000D81021EA0001C3F8D810D3F8002122EA20
:1061F0000002C3F80021D3F8003170470044025870
:1062000070B5D0E9244300224FF0FF359E6804EBBF
:1062100042135101D3F80009002805DAD3F8000928
:1062200040F08040C3F80009D3F8000B002805DADD
:10623000D3F8000B40F08040C3F8000B0132631824
:106240009642C3F80859C3F8085BE0D24FF0011337
:10625000C4F81C3870BD0000890141F020010161C3
:1062600003699B06FCD41220FFF7D2B910B50A4C83
:106270002046FEF75FFE094BC4F89030084BC4F887
:106280009430084C2046FEF755FE074BC4F890307A
:10629000064BC4F8943010BD608500200000084013
:1062A0007C7B0008FC85002000000440887B0008FF
:1062B00070B503780546012B5CD1434BD0F8904074
:1062C000984258D1414B0E216520D3F8D82042F096
:1062D0000062C3F8D820D3F8002142F00062C3F86E
:1062E0000021D3F80021D3F8802042F00062C3F8E7
:1062F0008020D3F8802022F00062C3F88020D3F8F9
:106300008030FEF793FA324BE360324BC4F800382A
:106310000023D5F89060C4F8003EC02323604FF4FA
:106320000413A3633369002BFCDA01230C203361CF
:10633000FFF76EF93369DB07FCD41220FFF768F929
:106340003369002BFCDA00262846A660FFF758FFC9
:106350006B68C4F81068DB68C4F81468C4F81C687B
:1063600083BB1D4BA3614FF0FF336361A36843F010
:106370000103A36070BD194B9842C9D1134B4FF074
:106380008060D3F8D82042F00072C3F8D820D3F848
:10639000002142F00072C3F80021D3F80021D3F8A5
:1063A000802042F00072C3F88020D3F8802022F0D1
:1063B0000072C3F88020D3F88030FFF70FFF0E2162
:1063C0004D209EE7064BCDE7608500200044025833
:1063D0004014004003002002003C30C0FC85002037
:1063E000083C30C0F8B5D0F89040054600214FF089
:1063F00000662046FFF730FFD5F8941000234FF0D9
:1064000001128F684FF0FF30C4F83438C4F81C28EC
:1064100004EB431201339F42C2F80069C2F8006BDB
:10642000C2F80809C2F8080BF2D20B68D5F8902020
:10643000C5F89830636210231361166916F01006D0
:10644000FBD11220FFF7E4F8D4F8003823F4FE6300
:10645000C4F80038A36943F4402343F01003A36158
:106460000923C4F81038C4F814380B4BEB604FF014
:10647000C043C4F8103B094BC4F8003BC4F8106992
:10648000C4F80039D5F8983003F1100243F48013B2
:10649000C5F89820A362F8BD587B00084080001022
:1064A000D0F8902090F88A10D2F8003823F4FE63D8
:1064B00043EA0113C2F80038704700002DE9F843A1
:1064C00000EB8103D0F890500C468046DA680FFA52
:1064D00081F94801166806F00306731E022B05EBCE
:1064E00041134FF0000194BFB604384EC3F8101B9F
:1064F0004FF0010104F1100398BF06F1805601FA34
:1065000003F3916998BF06F5004600293AD0578AEF
:1065100004F15801374349016F50D5F81C180B435B
:106520000021C5F81C382B180127C3F81019A74003
:106530005369611E9BB3138A928B9B08012A88BF03
:106540005343D8F89820981842EA034301F14002D7
:106550002146C8F89800284605EB82025360FFF7F1
:106560007BFE08EB8900C3681B8A43EA84534834E6
:106570001E4364012E51D5F81C381F43C5F81C7802
:10658000BDE8F88305EB4917D7F8001B21F400415B
:10659000C7F8001BD5F81C1821EA0303C0E704F173
:1065A0003F030B4A2846214605EB83035A60FFF759
:1065B00053FE05EB4910D0F8003923F40043C0F82E
:1065C0000039D5F81C3823EA0707D7E70080001008
:1065D00000040002D0F894201268C0F89820FFF759
:1065E0000FBE00005831D0F8903049015B5813F4C9
:1065F000004004D013F4001F0CBF0220012070479C
:106600004831D0F8903049015B5813F4004004D071
:1066100013F4001F0CBF02200120704700EB810122
:10662000CB68196A0B6813604B68536070470000B1
:1066300000EB810330B5DD68AA691368D36019B92E
:10664000402B84BF402313606B8A1468D0F89020DD
:106650001C4402EB4110013C09B2B4FBF3F4634368
:10666000033323F0030343EAC44343F0C043C0F8B9
:10667000103B2B6803F00303012B0ED1D2F808382E
:1066800002EB411013F4807FD0F8003B14BF43F0BD
:10669000805343F00053C0F8003B02EB4112D2F8A4
:1066A000003B43F00443C2F8003B30BD2DE9F0410C
:1066B000D0F8906005460C4606EB4113D3F8087BF2
:1066C0003A07C3F8087B08D5D6F814381B0704D559
:1066D00000EB8103DB685B689847FA071FD5D6F8A3
:1066E0001438DB071BD505EB8403D968CCB98B695B
:1066F000488A5A68B2FBF0F600FB16228AB918687D
:10670000DA6890420DD2121AC3E90024302383F3D1
:10671000118821462846FFF78BFF84F31188BDE8D6
:10672000F081012303FA04F26B8923EA02036B81EF
:10673000CB68002BF3D021462846BDE8F04118472E
:1067400000EB81034A0170B5DD68D0F890306C69C8
:106750002668E66056BB1A444FF40020C2F81009C0
:106760002A6802F00302012A0AB20ED1D3F80808FF
:1067700003EB421410F4807FD4F8000914BF40F0FA
:10678000805040F00050C4F8000903EB4212D2F8E8
:10679000000940F00440C2F800090122D3F834088F
:1067A00002FA01F10143C3F8341870BD19B9402E43
:1067B00084BF4020206020681A442E8A8419013C3E
:1067C000B4FBF6F440EAC44040F00050C6E70000D5
:1067D0002DE9F843D0F8906005460C464F0106EBD2
:1067E0004113D3F8088918F0010FC3F808891CD0A9
:1067F000D6F81038DB0718D500EB8103D3F80CC0AE
:10680000DCF81430D3F800E0DA68964530D2A2EB19
:106810000E024FF000091A60C3F80490302383F38E
:106820001188FFF78DFF89F3118818F0800F1DD0B4
:10683000D6F834380126A640334217D005EB84033E
:106840000134D5F89050D3F80CC0E4B22F44DCF8F2
:10685000142005EB0434D2F800E05168714514D3DC
:10686000D5F8343823EA0606C5F83468BDE8F8835D
:10687000012303FA01F2038923EA02030381DCF80E
:106880000830002BD1D09847CFE7AEEB0103BCF81E
:106890001000834228BF0346D7F8180980B2B3EB33
:1068A000800FE3D89068A0F1040959F8048FC4F868
:1068B0000080A0EB09089844B8F1040FF5D81844FB
:1068C0000B4490605360C8E72DE9F84FD0F8905022
:1068D00004466E69AB691E4016F480586E6103D0A1
:1068E000BDE8F84FFEF796BB002E12DAD5F8003E51
:1068F0009B0705D0D5F8003E23F00303C5F8003E02
:10690000D5F80438204623F00103C5F80438FEF713
:10691000AFFB370505D52046FFF772FC2046FEF792
:1069200095FBB0040CD5D5F8083813F0060FEB68CA
:1069300023F470530CBF43F4105343F4A053EB60A3
:1069400031071BD56368DB681BB9AB6923F008030B
:10695000AB612378052B0CD1D5F8003E9A0705D002
:10696000D5F8003E23F00303C5F8003E2046FEF7AD
:106970007FFB6368DB680BB120469847F30200F1A8
:10698000BA80B70226D5D4F8909000274FF0010ABC
:1069900009EB4712D2F8003B03F44023B3F5802FF4
:1069A00011D1D2F8003B002B0DDA62890AFA07F305
:1069B00022EA0303638104EB8703DB68DB6813B11E
:1069C0003946204698470137D4F89430FFB29B6887
:1069D0009F42DDD9F00619D5D4F89000026AC2F3BF
:1069E0000A1702F00F0302F4F012B2F5802F00F044
:1069F000CA80B2F5402F09D104EB8303002200F5D1
:106A00008050DB681B6A974240F0B0803003D5F8B5
:106A1000185835D5E90303D500212046FFF746FE77
:106A2000AA0303D501212046FFF740FE6B0303D5DF
:106A300002212046FFF73AFE2F0303D5032120460B
:106A4000FFF734FEE80203D504212046FFF72EFEAF
:106A5000A90203D505212046FFF728FE6A0203D5C7
:106A600006212046FFF722FE2B0203D507212046F0
:106A7000FFF71CFEEF0103D508212046FFF716FEA5
:106A8000700340F1A780E90703D500212046FFF7F6
:106A90009FFEAA0703D501212046FFF799FE6B0749
:106AA00003D502212046FFF793FE2F0703D50321CC
:106AB0002046FFF78DFEEE0603D504212046FFF7A2
:106AC00087FEA80603D505212046FFF781FE69064B
:106AD00003D506212046FFF77BFE2A0603D50721B2
:106AE0002046FFF775FEEB0574D520460821BDE86A
:106AF000F84FFFF76DBED4F890904FF0000B4FF0B9
:106B0000010AD4F894305FFA8BF79B689F423FF6F6
:106B100038AF09EB4713D3F8002902F44022B2F54D
:106B2000802F20D1D3F80029002A1CDAD3F80029BD
:106B300042F09042C3F80029D3F80029002AFBDB79
:106B40003946D4F89000FFF787FB22890AFA07F349
:106B500022EA0303238104EB8703DB689B6813B1FC
:106B60003946204698470BF1010BCAE7910701D13E
:106B7000D0F80080072A02F101029CBF03F8018BC4
:106B80004FEA18283FE704EB830300F58050DA68EA
:106B9000D2F818C0DCF80820DCE9001CA1EB0C0CD2
:106BA00000218F4208D1DB689B699A683A449A6059
:106BB0005A683A445A6029E711F0030F01D1D0F81E
:106BC00000808C4501F1010184BF02F8018B4FEA7E
:106BD0001828E6E7BDE8F88F08B50348FFF774FE0C
:106BE000BDE80840FDF7E6BC6085002008B5034815
:106BF000FFF76AFEBDE80840FDF7DCBCFC8500201D
:106C0000D0F8903003EB4111D1F8003B43F400136E
:106C1000C1F8003B70470000D0F8903003EB411101
:106C2000D1F8003943F40013C1F80039704700006F
:106C3000D0F8903003EB4111D1F8003B23F400135E
:106C4000C1F8003B70470000D0F8903003EB4111D1
:106C5000D1F8003923F40013C1F80039704700005F
:106C600030B50433039C0172002104FB0325C1608D
:106C7000C0E90653049B0363059BC0E90000C0E91B
:106C80000422C0E90842C0E90A11436330BD000094
:106C90000022416AC260C0E90411C0E90A226FF013
:106CA0000101FEF725BD0000D0E90432934201D175
:106CB000C2680AB9181D704700207047036919603F
:106CC0000021C2680132C260C269134482699342E2
:106CD000036124BF436A0361FEF7FEBC38B5044676
:106CE0000D46E3683BB162690020131D1268A36280
:106CF0001344E36207E0237A33B929462046FEF7BE
:106D0000DBFC0028EDDA38BD6FF00100FBE7000086
:106D1000C368C269013BC3604369134482699342FB
:106D2000436124BF436A436100238362036B03B161
:106D30001847704770B53023044683F31188866A7C
:106D40003EB9FFF7CBFF054618B186F311882846F8
:106D500070BDA36AE26A13F8015B9342A36202D397
:106D60002046FFF7D5FF002383F31188EFE70000EB
:106D70002DE9F84F04460E46174698464FF0300965
:106D800089F311880025AA46D4F828B0BBF1000F7A
:106D900009D141462046FFF7A1FF20B18BF31188AE
:106DA0002846BDE8F88FD4E90A12A7EB050B521A62
:106DB000934528BF9346BBF1400F1BD9334601F1E1
:106DC000400251F8040B914243F8040BF9D1A36A35
:106DD000403640354033A362D4E90A239A4202D3B5
:106DE0002046FFF795FF8AF31188BD42D8D289F378
:106DF0001188C9E730465A46FAF746FFA36A5E444F
:106E00005D445B44A362E7E710B5029C0433017262
:106E100003FB0421C460C0E906130023C0E90A3360
:106E2000039B0363049BC0E90000C0E90422C0E99E
:106E30000842436310BD0000026A6FF00101C260A6
:106E4000426AC0E904220022C0E90A22FEF750BCCF
:106E5000D0E904239A4201D1C26822B9184650F8F9
:106E6000043B0B60704700231846FAE7C368002113
:106E7000C2690133C3604369134482699342436129
:106E800024BF436A4361FEF727BC000038B50446BF
:106E90000D46E3683BB1236900201A1DA262E26936
:106EA0001344E36207E0237A33B929462046FEF70C
:106EB00003FC0028EDDA38BD6FF00100FBE70000AD
:106EC00003691960C268013AC260C26913448269E9
:106ED0009342036124BF436A036100238362036B0F
:106EE00003B118477047000070B530230D460446C3
:106EF000114683F31188866A2EB9FFF7C7FF10B1D8
:106F000086F3118870BDA36A1D70A36AE26A01331B
:106F10009342A36204D3E16920460439FFF7D0FF0E
:106F2000002080F31188EDE72DE9F84F04460D4667
:106F3000904699464FF0300A8AF311880026B346EE
:106F4000A76A4FB949462046FFF7A0FF20B187F353
:106F500011883046BDE8F88FD4E90A073A1AA8EB41
:106F60000607974228BF1746402F1BD905F140035B
:106F700055F8042B9D4240F8042BF9D1A36A403602
:106F80004033A362D4E90A239A4204D3E16920463C
:106F90000439FFF795FF8BF311884645D9D28AF360
:106FA0001188CDE729463A46FAF76EFEA36A3D44BA
:106FB0003E443B44A362E5E7D0E904239A4217D15B
:106FC000C3689BB1836A8BB1043B9B1A0ED01360DC
:106FD000C368013BC360C3691A4483699A42026172
:106FE00024BF436A0361002383620123184670476C
:106FF0000023FBE700F024B9014B586A704700BF3B
:10700000000C0040034B002258631A610222DA6030
:10701000704700BF000C0040014B0022DA6070474F
:10702000000C0040014B5863704700BF000C00404B
:10703000FEE7000070B51B4B0025044686B0586083
:107040000E4685620163FDF78DFA04F11003A56019
:10705000E562C4E904334FF0FF33C4E90044C4E9F6
:107060000635FFF7C9FF2B46024604F134012046DE
:10707000C4E9082380230C4A2565FEF7D3FA0123CF
:107080000A4AE06000920375684672680192B2682D
:10709000CDE90223064BCDE90435FEF7EBFA06B045
:1070A00070BD00BF086A0020947B0008997B00082F
:1070B00031700008024AD36A1843D062704700BF9B
:1070C000A06700204B6843608B688360CB68C36017
:1070D0000B6943614B6903628B6943620B68036010
:1070E0007047000008B53C4B40F2FF713B48D3F8B5
:1070F00088200A43C3F88820D3F8882022F4FF624E
:1071000022F00702C3F88820D3F88820D3F8E020C3
:107110000A43C3F8E020D3F808210A43C3F8082142
:107120002F4AD3F808311146FFF7CCFF00F58060F5
:1071300002F11C01FFF7C6FF00F5806002F1380183
:10714000FFF7C0FF00F5806002F15401FFF7BAFFBE
:1071500000F5806002F17001FFF7B4FF00F5806078
:1071600002F18C01FFF7AEFF00F5806002F1A8018B
:10717000FFF7A8FF00F5806002F1C401FFF7A2FF4E
:1071800000F5806002F1E001FFF79CFF00F58060F0
:1071900002F1FC01FFF796FF02F58C7100F58060AB
:1071A000FFF790FF00F014F90E4BD3F8902242F055
:1071B0000102C3F89022D3F8942242F00102C3F8EE
:1071C00094220522C3F898204FF06052C3F89C2007
:1071D000054AC3F8A02008BD004402580000025828
:1071E000A07B000800ED00E01F00080308B500F0D8
:1071F000D1FAFEF7CBF90F4BD3F8DC2042F0400276
:10720000C3F8DC20D3F8042122F04002C3F80421A3
:10721000D3F80431084B1A6842F008021A601A6861
:1072200042F004021A60FEF72FFFBDE80840FEF7A7
:107230004BBC00BF004402580018024870470000D1
:10724000114BD3F8E82042F00802C3F8E820D3F845
:10725000102142F00802C3F810210C4AD3F8103173
:10726000D36B43F00803D363C722094B9A624FF0F4
:10727000FF32DA6200229A615A63DA605A600122B0
:107280005A611A60704700BF004402580010005C49
:10729000000C0040094A08B51169D3680B40D9B207
:1072A0009B076FEA0101116107D5302383F3118831
:1072B000FEF792F9002383F3118808BD000C00400B
:1072C000064BD3F8DC200243C3F8DC20D3F80421BA
:1072D0001043C3F80401D3F8043170470044025846
:1072E0003A4B4FF0FF31D3F8802062F00042C3F8F0
:1072F0008020D3F8802002F00042C3F88020D3F829
:107300008020D3F88420C3F88410D3F8842000228E
:10731000C3F88420D3F88400D86F40F0FF4040F4D5
:10732000FF0040F4DF4040F07F00D867D86F20F0C6
:10733000FF4020F4FF0020F4DF4020F07F00D867FA
:10734000D86FD3F888006FEA40506FEA5050C3F806
:107350008800D3F88800C0F30A00C3F88800D3F887
:107360008800D3F89000C3F89010D3F89000C3F8C9
:107370009020D3F89000D3F89400C3F89410D3F879
:107380009400C3F89420D3F89400D3F89800C3F87D
:107390009810D3F89800C3F89820D3F89800D3F841
:1073A0008C00C3F88C10D3F88C00C3F88C20D3F871
:1073B0008C00D3F89C00C3F89C10D3F89C10C3F841
:1073C0009C20D3F89C3000F0B9B900BF00440258AB
:1073D00008B50122534BC3F80821534BD3F8F420CE
:1073E00042F00202C3F8F420D3F81C2142F002025A
:1073F000C3F81C210222D3F81C314C4BDA605A68C6
:107400009104FCD54A4A1A6001229A60494ADA601E
:1074100000221A614FF440429A61444B9A699204E7
:10742000FCD51A6842F480721A603F4B1A6F12F44E
:10743000407F04D04FF480321A6700221A671A681E
:1074400042F001021A60384B1A685007FCD500223E
:107450001A611A6912F03802FBD1012119604FF04C
:10746000804159605A67344ADA62344A1A611A68AC
:1074700042F480321A602C4B1A689103FCD51A68CA
:1074800042F480521A601A689204FCD52C4A2D49A5
:107490009A6200225A63196301F57C01DA6301F5EF
:1074A000E77199635A64284A1A64284ADA621A68AA
:1074B00042F0A8521A601C4B1A6802F02852B2F12E
:1074C000285FF9D148229A614FF48862DA6140223C
:1074D0001A621F4ADA641F4A1A651F4A5A651F4A10
:1074E0009A6532231E4A1360136803F00F03022BC0
:1074F000FAD10D4A136943F003031361136903F0D2
:107500003803182BFAD14FF00050FFF7D9FE4FF097
:107510008040FFF7D5FE4FF00040BDE80840FFF780
:10752000CFBE00BF008000510044025800480258FE
:1075300000C000F0020000010000FF010088900878
:107540003220600063020901470E0508DD0BBF0110
:1075500020000020000001100910E00000010110CF
:10756000002000524FF0B04208B5D2F8883003F046
:107570000103C2F8883023B1044A13680BB1506884
:107580009847BDE80840FDF715B800BFB086002059
:107590004FF0B04208B5D2F8883003F00203C2F8C9
:1075A000883023B1044A93680BB1D0689847BDE88E
:1075B0000840FCF7FFBF00BFB08600204FF0B0428C
:1075C00008B5D2F8883003F00403C2F8883023B13C
:1075D000044A13690BB150699847BDE80840FCF7AD
:1075E000E9BF00BFB08600204FF0B04208B5D2F826
:1075F000883003F00803C2F8883023B1044A936945
:107600000BB1D0699847BDE80840FCF7D3BF00BF75
:10761000B08600204FF0B04208B5D2F8883003F0B1
:107620001003C2F8883023B1044A136A0BB1506AC0
:107630009847BDE80840FCF7BDBF00BFB0860020FA
:107640004FF0B04310B5D3F8884004F47872C3F813
:107650008820A30604D5124A936A0BB1D06A9847D2
:10766000600604D50E4A136B0BB1506B9847210688
:1076700004D50B4A936B0BB1D06B9847E20504D548
:10768000074A136C0BB1506C9847A30504D5044A04
:10769000936C0BB1D06C9847BDE81040FCF78ABFE3
:1076A000B08600204FF0B04310B5D3F8884004F402
:1076B0007C42C3F88820620504D5164A136D0BB1CD
:1076C000506D9847230504D5124A936D0BB1D06DC8
:1076D0009847E00404D50F4A136E0BB1506E9847DB
:1076E000A10404D50B4A936E0BB1D06E9847620487
:1076F00004D5084A136F0BB1506F9847230404D583
:10770000044A936F0BB1D06F9847BDE81040FCF767
:1077100051BF00BFB086002008B50348FDF700F850
:10772000BDE80840FCF746BF3463002008B5FFF70A
:10773000B1FDBDE80840FCF73DBF0000062108B5DB
:107740000846FDF773F806210720FDF76FF80621BC
:107750000820FDF76BF806210920FDF767F80621E0
:107760000A20FDF763F806211720FDF75FF80621D0
:107770002820FDF75BF809217A20FDF757F807214B
:107780003220FDF753F80C215220BDE80840FDF7E8
:107790004DB8000008B5FFF7A3FD00F00DF8FDF7A8
:1077A000EDF9FDF7C5FBFDF797FAFFF747FDBDE8DB
:1077B0000840FFF71FBC00000023054A19460133AB
:1077C000102BC2E9001102F10802F8D1704700BF86
:1077D000B08600200B460146184600F003B80000B2
:1077E00000F00EB810B5054C13462CB10A46014600
:1077F0000220AFF3008010BD2046FCE7000000002F
:10780000024B01461868FEF757BB00BF6C220020F0
:1078100010B501390244904201D1002005E00378FF
:1078200011F8014FA34201D0181B10BD0130F2E73F
:107830002DE9F041A3B1C91A17780144044603F1B8
:10784000FF3C8C42204601D9002009E00578BD426A
:1078500004F10104F5D10CEB0405D618A54201D1C1
:10786000BDE8F08115F8018D16F801EDF045F5D071
:10787000E7E70000034611F8012B03F8012B002A6B
:10788000F9D170476F72672E6172647570696C6FA1
:10789000742E437562654F72616E67652D706572F7
:1078A0006970680053544D333248373F3F3F0053AF
:1078B000544D3332483733782F3732780053544D94
:1078C0003332483734332F3735332F3735300000D4
:1078D00001105A00031059000120580003205600DF
:1078E00040A2E4F1646891060041A3E5F265699263
:1078F0000700000043414E464449666163653A20F3
:107900004D6573736167652052414D204F766572F6
:10791000666C6F77210000004261642043414E494C
:107920006661636520696E6465782E000001000061
:107930000001FF0000A0004000A400400000000083
:1079400000000000DD2C0008B525000811340008F7
:10795000AD25000825260008352A00089D270008C7
:10796000ED250008F1250008C9250008B12500080B
:10797000F5290008D525000879350008E12500081B
:10798000C929000800960000000000000000000067
:1079900000000000000000000000000000000000E7
:1079A0003D4B0008294B0008654B0008514B00086F
:1079B0005D4B0008494B0008354B0008214B00087F
:1079C000714B000800000000554C0008414C0008B5
:1079D0007D4C0008694C0008754C0008614C00089B
:1079E0004D4C0008394C0008894C0008000000008C
:1079F000010000000000000063300000F87900087A
:107A0000F8670020086A00204172647550696C6F45
:107A1000740025424F415244252D424C00255345C8
:107A20005249414C25000000020000000000000007
:107A3000754E0008E54E000840004000B882002066
:107A4000C8820020020000000000000003000000C7
:107A5000000000002D4F0008000000001000000092
:107A6000D88200200000000001000000000000009B
:107A70006085002001010200655A00087559000860
:107A8000115A0008F559000843000000907A0008D8
:107A900009024300020100C0320904000001020291
:107AA0000100052400100105240100010424020244
:107AB0000524060001070582030800FF09040100F0
:107AC000020A0000000705010240000007058102CC
:107AD0004000000012000000DC7A000812011001D2
:107AE0000200004009124157000201020301000098
:107AF0000403090425424F415244250030313233FA
:107B00003435363738394142434445460000000099
:107B10000000002000000200020000000001003010
:107B20000000000008000000000000240000080021
:107B3000040000000004000000FC0000020000003F
:107B40000000043000800000080000000000003841
:107B50000000010001000000000000008950000842
:107B600041530008ED530008400040009886002073
:107B70009886002001000000A886002080000000F8
:107B8000400100000800000000010000001000009B
:107B9000080000006D61696E0069646C650000009A
:107BA0000000802A00000000AAAAAAAA000000245F
:107BB000FFFF00000000000000A00A0000210002FA
:107BC00000000000AAAAAAAA00000000FFFF00000F
:107BD000000000090000090014000054000000002B
:107BE000AAAAAAAA14000054FFFF00000000000087
:107BF000000000000A40100000000000AAAA8AAAA3
:107C000000401000FFFF000099000000000000008D
:107C10000081020000000000AAAAAAAA00410100F7
:107C2000FFFF0000000000700700000000000000DF
:107C300000000000AAAAAAAA00000000FFFF00009E
:107C40000000000000000000000000000000000034
:107C5000AAAAAAAA00000000FFFF0000000000007E
:107C6000000000000000000000000000AAAAAAAA6C
:107C700000000000FFFF0000000000000000000006
:107C80000000000000000000AAAAAAAA000000004C
:107C9000FFFF0000000000000000000000000000E6
:107CA00000000000AAAAAAAA00000000FFFF00002E
:107CB00000000000000000000000000000000000C4
:107CC000AAAAAAAA00000000FFFF0000000000000E
:107CD000000000004C86FF7F010000000000000053
:107CE000780500000000000000001E0000000000F9
:107CF000FE2A0100D2040000FF000000106A0020EC
:107D00003463002000000000A47800088304000011
:107D1000AF78000850040000BD780008009600000D
:107D200000000800960000000008000004000000A9
:107D3000F07A0008000000000000000000000000D1
:107D40000000000000000000000000007022002081
:107D50000000000000000000000000000000000023
:107D60000000000000000000000000000000000013
:107D70000000000000000000000000000000000003
:107D800000000000000000000000000000000000F3
:107D900000000000000000000000000000000000E3
:107DA00000000000000000000000000000000000D3
:00000001FF
